S0200000557362537069446F6E676C654B4C32355A5F4744333030302E7372656350
S1130000000000202908000089080000A908000059
S11300109108000091080000910800009108000078
S11300209108000091080000910800009108000068
S1130030910800009108000091080000C52A000002
S11300409108000091080000910800009108000048
S11300509108000091080000910800009108000038
S11300609108000091080000910800009108000028
S11300709108000091080000910800009108000018
S11300809108000091080000910800009108000008
S113009091080000910800009108000091080000F8
S11300A0E961000091080000910800009108000037
S11300B09108000091080000A90F000091080000B9
S113080080B500AF054A064BD31A054A101C0021D7
S11308101A1C06F05EF9BD4680BDC046000A0020E1
S11308200000002000F000F806F02AFD00F040F877
S1130830FFF7E6FF06F0FCFC06F098FC06F02EFD40
S1130840044B0020191C00F0F7F9031C181C06F0D7
S11308501BF9C0460000002080B582B000AF78606C
S1130860FEE7C04680B500AF044B044A1278D2B20A
S113087020210A43D2B21A70BD4680BD00F0074061
S113088080B500AFBD4680BD80B500AFBD4680BD1C
S113089080B582B000AF034AFB1D12781A70BD46C2
S11308A002B080BD04ED00E080B500AFBD4680BD60
S11308B080B500AF034A88235B010021D150BD46B7
S11308C080BDC0460070044080B582B000AF021CF9
S11308D0FB1D1A70064B181C0021282206F0F9F89B
S11308E000F078F8031C181CBD4602B080BDC04659
S11308F02804002080B584B000AF78607B68002BAA
S113090001D1FF233DE07B681B68013301D1FF2344
S113091037E03B1C0F3300221A7023E000F0B4F8D8
S11309203B1C0F331B78194ADB00D31804331B68B4
S1130930002B0ED13B1C0F331B78DA00134BD2185B
S11309407B68101C191C082206F0BAF800F080F825
S11309500DE000F07DF83B1C0F333A1C0F32127887
S113096001321A703B1C0F331B78042BD6D93B1C65
S11309700F331B78052B01D1FE2302E03B1C0F3300
S11309801B78181CBD4604B080BDC0462804002056
S113099080B582B000AF021CFB1D1A70FB1D1B78D2
S11309A0042B01D9FF230EE000F06EF8FB1D1B7829
S11309B0DA00074BD318181C0021082206F089F826
S11309C000F046F80023181CBD4602B080BDC046A6
S11309D02804002080B500AF184A1849184BCB589A
S11309E0802109041943164BD150164B042252425C
S11309F01A60144A80235B001349D150114A84239E
S1130A005B0002214942D1500E4A84235B0003213A
S1130A104942D1500B4A86235B000121D1500B4A35
S1130A20C0235B008021C903D150084B8022D2032C
S1130A301A600023181CBD4680BDC04600700440E7
S1130A403C10000000700340C05D000000E100E0C5
S1130A5080B500AF0B4A0B4984235B00CB580121BE
S1130A60194384235B00D150064A064984235B0062
S1130A70CB580221194384235B00D150C046BD46A4
S1130A8080BDC0460070034080B500AF0D4A0D49DB
S1130A9084235B00CB580121181C8843011C842348
S1130AA05B00D150074A074984235B00CB580221DD
S1130AB0181C8843011C84235B00D150C046BD46EA
S1130AC080BDC0460070034080B584B000AF2A4AA0
S1130AD086235B00D2580123134047D0264A264977
S1130AE086235B00CB580121194386235B00D15038
S1130AF0FFF7CAFF214AC0235B008021C903D150FC
S1130B001E4B8022D2031A603B1C0F3300221A7042
S1130B1027E03B1C0F331B78DA00194BD318BB605A
S1130B20BB685B68002B14D0BB681B685A1EBB688B
S1130B301A60BB681B68002B0CD1BB685B687B60C8
S1130B403B1C0F331B78181CFFF722FF7B68984768
S1130B5000E0C0463B1C0F333A1C0F3212780132BE
S1130B601A703B1C0F331B78042BD2D9FFF770FF8C
S1130B70BD4604B080BDC0460070034000E100E003
S1130B802804002080B582B000AF00237B60244A93
S1130B902349244BCB58802109011943214BD150BF
S1130BA0214B214AD168214A0A40DA601E4B1E4A71
S1130BB0D268A021C9000A43DA601D4B1C4A12788E
S1130BC0D2B202218A43D2B21A70154A1449194B7F
S1130BD0CB5880211943174BD150154B144A5278E6
S1130BE0D2B201210A43D2B25A70114B104A127A7E
S1130BF0D2B20E218A43D2B21A720D4B0C4A127A27
S1130C00D2B204210A43D2B21A72094B084A1278AA
S1130C10D2B202210A43D2B21A70BD4602B080BDDC
S1130C20007004403810000000B00440FFF8FFFFDB
S1130C30004006400410000080B500AF00F0A4F9A5
S1130C40002000F0E5F800F017F800F021F901F0B9
S1130C5013FAFFF797FF01F03DFE01F03FFD01F0AD
S1130C605FFD0020FFF730FE00F0B0FBFFF7FAFD58
S1130C7000F0D4FBFAE7C04680B500AF564A5649A7
S1130C80564BCB58F82189011943544BD150544B3E
S1130C90802252005A61524B802252001A64504BF7
S1130CA0802252005A644F4B802252001A624E4BEB
S1130CB04D4A52694D490A435A614D4B4C4A526957
S1130CC0802149000A435A61454B802252001A612F
S1130CD0454B454A526910218A435A61404B404A68
S1130CE0126903210A431A613D4B3D4A126990215E
S1130CF009030A431A613F4AA0230821D150384A04
S1130D00A0231021D1503C4AC0235B008021C90597
S1130D10D150394B8022D2051A60364B80225200C2
S1130D205A62364B354A5269802189000A435A6116
S1130D30334B802252005A61324B324A526920218D
S1130D400A435A61304B80225200DA602F4B2F4AFB
S1130D50526908210A435A612B4B802252001A61BE
S1130D602A4B2A4A526910210A435A61264B80228F
S1130D7052005A61254B254A526920210A435A617F
S1130D80214B802252009A60204B204A5269042150
S1130D900A435A61134B80225200DA62144B144AFC
S1130DA05269802109010A435A610E4B8022520084
S1130DB09A620F4B0E4A52698021C9000A435A6154
S1130DC0114B802252001A60104B104A52690121C3
S1130DD00A435A61BD4680BD0070044038100000CB
S1130DE00090044000A0044000F00F4020000300E5
S1130DF040F00F4000B0044000E100E080F00F40FC
S1130E0000C00440C0F00F4000D0044000F10F4087
S1130E1080B582B000AF021CFB1D1A70FB1D1B784D
S1130E20002B27D1154A1549154BCB58A021C902CF
S1130E301943134BD150114A1049124BCB588021FE
S1130E40C90219430F4BD1500F4A86235B0040213E
S1130E50D1540A4B094A1268802109060A431A60D0
S1130E600A4AC0235B0080214904D150074B8022E9
S1130E7052041A60BD4602B080BDC04600700440F2
S1130E8004100000341000000020074000E100E0DE
S1130E9080B500AF2C4A2C492C4BCB588021C9007B
S1130EA019432A4BD1502A4B802252009A64294B71
S1130EB0284A52688021C9020A435A60254B254AB0
S1130EC052698021C9020A435A611F4A1E491F4BB5
S1130ED0CB588021C90019431C4BD1501C4B802294
S1130EE05200DA641B4B1B4A5268802109030A43EF
S1130EF05A60184B174A5269802109030A435A6100
S1130F00114A1149114BCB588021490119430F4B08
S1130F10D150114B802252005A60104B02225A6069
S1130F200E4B0E4A526902210A435A61094B802230
S1130F30D2029A60074B802212035A60074B0222A6
S1130F405A60BD4680BDC0460070044038100000A1
S1130F5000A0044040F00F4000C00440C0F00F4027
S1130F6080B500AFBD4680BD80B584B000AF021C23
S1130F70FB1D1A703B1C0F3300221A70FFF7F0FFA1
S1130F80BD4604B080BDC04680B500AF034A0449E5
S1130F90044BD15000F0A0F9BD4680BD00E000E054
S1130FA000000000080D000080B500AF0F4AC02308
S1130FB05B008021C905D1500C4B8022D2051A60F8
S1130FC072B60B4AA023D258102313400BD0094BFE
S1130FD01B78DBB202221343DAB2064B1A70044ABE
S1130FE0A0231021D15062B6BD4680BD00E100E0CF
S1130FF0009004405004002080B500AF074A074920
S1131000D1231B01CB580421181C8843011CD12374
S11310101B01D15030BFBD4680BDC04600E000E09A
S113102080B500AF064A0649D1231B01CB580421E1
S11310301943D1231B01D15030BFBD4680BDC046EA
S113104000E000E080B500AFFFF7D6FFBD4680BDED
S113105080B582B000AF0B4B0A4A5278D2B2072156
S11310608A43D2B25A70074B064A5278D2B25A70A7
S1131070044B5B78DBB27B60FFF7D2FFBD4602B066
S113108080BDC04600E0074080B584B000AF021CBC
S1131090FB1D1A70264BDB78DBB21A1C7F2313402E
S11310A0042B01D114233EE0214B20221A70FB1D96
S11310B0FA1D117801220A401A701D4B1C4A5278FD
S11310C0D2B260218A43D2B25A70194B184A52786C
S11310D0D2B240210A43D2B25A700023FB6009E025
S11310E0144B9B78DBB21A1C0423134006D0FB6814
S11310F00133FB60FB68092BF2DD00E0C0460D4BB9
S11311009B78DBB21A1C0423134001D024230AE089
S1131110074BDB78DBB21A1C7F231340042B01D16D
S1131120042300E00023181CBD4604B080BDC04663
S113113000E0074000D0074080B582B000AF0E4BFE
S113114020221A700C4B0C4A5278D2B207218A43DF
S1131150D2B25A70084B084A5278D2B202210A43DA
S1131160D2B25A70044B5B78DBB27B60FFF758FF56
S1131170BD4602B080BDC04600E0074080B582B0E5
S113118000AF0E4B08221A700C4B0C4A5278D2B2A4
S113119007218A43D2B25A70084B084A5278D2B215
S11311A003210A43D2B25A70044B5B78DBB27B60F2
S11311B0FFF736FFBD4602B080BDC04600E00740E1
S11311C080B582B000AF0F4B02221A700D4B0D4A4E
S11311D05278D2B207218A43D2B25A70094B094AD3
S11311E05278D2B204210A43D2B25A70054B032278
S11311F09A70044B9B78DBB27B60FFF711FFBD460E
S113120002B080BD00E0074080B582B000AF0F4B54
S113121002221A700D4B0D4A5278D2B207218A432A
S1131220D2B25A70094B094A5278D2B204210A4305
S1131230D2B25A70054B01229A70044B9B78DBB2F0
S11312407B60FFF7EDFEBD4602B080BD00E00740C5
S113125080B584B000AF021CFB1D1A700E4B022235
S11312601A700D4B0C4A5278D2B207218A43D2B27B
S11312705A70094B084A5278D2B204210A43D2B2B6
S11312805A70054B00229A70034B9B78DBB2FB60CB
S1131290BD4604B080BDC04600E0074080B500AF45
S11312A00B4B0B4A1278D1B23F220A40D2B21A70C9
S11312B0C046074B9B79DBB21A1C0C2313409B08D6
S11312C0032BF6D1034B80221A70BD4680BDC04665
S11312D0004006400050064080B500AF384A394B04
S11312E080214902D150364A3549364BCB588021AA
S11312F049051943334BD150334B25225A70324B95
S113130098221A70304B304AD278D1B21F220A4048
S1131310D2B2DA702C4B23221A712B4B18225A7139
S1131320C046294B9B79DBB21A1C10231340F8D119
S1131330C046254B9B79DBB21A1C0C231340082BA7
S1131340F7D1214B98221A701F4B25225A701E4B3D
S113135023221A711C4B58225A71C0461A4B9B798E
S1131360DBB21A1C0C231340082BF7D1C046164BD2
S11313709B79DBB21A1C40231340F8D0124B18227D
S11313801A70114B25225A700F4B23221A710E4BDF
S113139058225A71C0460C4B9B79DBB21A1C0C23A1
S11313A013400C2BF7D1084B074A5279D2B22021B3
S11313B00A43D2B25A710023181CBD4680BDC046F0
S11313C000700440441000000040064090B585B011
S11313D002AF0E4B00221A700D4B00221A7072B627
S11313E0FC1D0C4A0C4B012100910020111C002211
S11313F002F0E4F8031C2370FB1D1B78002B01D1C1
S113140062B600E0C046BD4603B090BD880000202F
S113141089000020A51A0000891B000080B500AFD8
S113142003F096FA064B1B78DBB2012B06D1054B71
S11314301B78DBB2012B01D100F006F8BD4680BD5C
S11314400400002000F0FF1F90B589B000AF3B1CE2
S1131450163300221A703B1C153300221A703B1CF1
S1131460143300221A703B1C133300221A703B1CE5
S1131470123300221A703B1C103300221A80DA4BFC
S11314801B78002B00D144E2D84B00221A700DE0E7
S1131490D64B1B78D54A1278D549895CD54AD154A4
S11314A0D24B1B780133DAB2D04B1A70CF4B1A7877
S11314B0CD4B1B789A42EBD3CB4B1A78CE4B1A7098
S11314C0C94B00221A70CA4B1B78092B32D1C94B65
S11314D0FA221A70C74B05225A70C64B03229A701F
S11314E0C44B0022DA70C34B00221A71C14B002294
S11314F05A71C04B00229A71BE4B0022DA713B1C18
S11315000F3308221A703B1C0F331B789BB2B94A65
S11315100020012102F02EF9031C1A1CB34B1A708F
S1131520B24B1B78002B00D0F3E1B44B8022D202E3
S11315305A60EEE1AE4B1B780E2B1ED13B1C0E33D2
S113154008221A703B1C0E331B789BB2A94A002058
S1131550012102F00FF9031C1A1CA44B1A70A34BAF
S11315601B78002B00D0D4E1A44B8022D2029A60D5
S1131570A24B802212035A60CBE19D4B1B78A04AF8
S113158012781340DAB29E4B1B789A4200D09DE049
S11315909B4B1A78974B1A70954B5A78954B5A7007
S11315A0934B5A78974B1B789A4244D13B1C0D338A
S11315B08F4AD2791A703B1C0D331B78072B2ED817
S11315C00023FB610023BB61FA239B00BB60002363
S11315D0FB610CE03B1C0D331B78181C01F05CF91B
S11315E0031CBA69D318BB61FB690133FB61FA6957
S11315F0BB689A42EED3B869B96805F0F5F9031CE3
S11316001A1CBB1D1A80BB1D1B88DAB2794B5A7198
S1131610BB1D1B881B0A9BB2DAB2764B1A71764B40
S11316201B78744A0020012102F0A4F8031C1A1C40
S11316306E4B1A706DE16E4B5A78734B1B789A425D
S113164025D17B1D08221A707B1D1B789BB2694A29
S11316500020012102F08EF8031C1A1C634B1A703F
S1131660634B1B791A06624B5B791B041A43604B6C
S11316709B791B021A435E4BDB7913431A1C634BA1
S11316801A60624B1B68181C01F03EF941E1584B8B
S11316905A785F4B1B789A4200D03AE1554B0022AE
S11316A01A715C4B1A6980235B02134002D0514BC0
S11316B001221A71504B1B784E4A0020012102F07E
S11316C059F8031C1A1C494B1A7022E1484B5978EB
S11316D03B1C163303220A401A70454B99783B1C75
S11316E0153307220A401A70414B19783B1C1433F6
S11316F07F220A401A703B1C13333A1C14321278AE
S1131700D2081A703A4B5A783B1C1233D2091A7019
S11317103B1C12331B78002B0CD13B1C16331B785B
S1131720181C00F047FD3B1C15331B78181C00F0F7
S1131730AFFD0BE03B1C16331B78181C00F0C8FEF1
S11317403B1C15331B78181C00F030FF3B1C17336F
S113175004221A70264B5B781A1C4023134000D0D5
S1131760BFE03B1C12331B78002B06D1204B5B7867
S11317700120191C00F0D0FD96E01D4B5B78012080
S1131780191C00F057FF8FE0194B5B781A1C2023BB
S113179013401AD13B1C12331B78002B0AD13B1C7B
S11317A017331B78124AD35CDB43DBB2181C00F0FE
S11317B0B3FC39E03B1C17331B780D4AD35CDB4385
S11317C0DBB2181C00F036FE2EE03B1C12331B78F3
S11317D0002B21D13B1C17331B78054AD35C181C02
S11317E000F09AFC20E0C046880000209000002011
S11317F008000020480000208900002040F00F402D
S1131800A0720000A1720000A37200008C000020EE
S1131810A272000080F00F403B1C17331B783F4A34
S1131820D35C181C00F006FE3C4B5B781A1C10239A
S113183013401AD13B1C12331B78002B0AD13B1CDA
S113184017331C7800F082FC031CDB43DAB2344B00
S11318501A5522E03B1C17331C7800F005FE031CCC
S1131860DB43DAB22E4B1A5517E03B1C12331B78BC
S1131870002B09D13B1C17331C7800F067FC031CB8
S11318801A1C274B1A5508E03B1C17331C7800F030
S1131890EBFD031C1A1C224B1A553B1C17333A1C34
S11318A01732127801321A703B1C17331A783B1C1A
S11318B013331B7804339A4200DA65E73B1C123376
S11318C01B78002B06D1154B5B780020191C00F007
S11318D023FD0EE0114B5B780020191C00F0AAFEDA
S11318E007E00E4BDA780D4B9B78101C191C00F0A6
S11318F01DF83B1D0B4A12781A703B1D1B789BB2D6
S1131900074A0020012101F035FF031C1A1C064B75
S11319101A70C046BD4609B090BDC04608000020FC
S113192048000020890000209000002080B582B08B
S113193000AF0A1CFB1D011C1970BB1D1A70FB1D96
S11319401A780123134007D0524B524A526880211F
S113195089000A435A6006E04E4B4E4A9268802141
S113196089000A439A60FB1D1A780223134006D0AB
S1131970494B494A526820210A435A6005E0464BC4
S1131980454A926820210A439A60FB1D1A78042371
S1131990134006D0414B414A526808210A435A6019
S11319A005E03E4B3D4A926808210A439A60FB1DBC
S11319B01A780823134006D0384B384A526810214D
S11319C00A435A6005E0354B344A926810210A43B1
S11319D09A60FB1D1A781023134006D02F4B2F4A10
S11319E0526820210A435A6005E02C4B2B4A926826
S11319F020210A439A60FB1D1A782023134006D045
S1131A00264B264A526804210A435A6005E0234BB8
S1131A10224A926804210A439A60FB1D1A784023E3
S1131A20134007D01E4B1E4A5268802109010A4305
S1131A305A6006E01A4B1A4A9268802109010A4347
S1131A409A60FB1D1B785BB2002B07DA144B144A17
S1131A5052688021C9000A435A6006E0104B104ABC
S1131A6092688021C9000A439A60BB1D1B785BB24F
S1131A70002B06DA094B094A526801210A435A60CD
S1131A8005E0064B054A926801210A439A60BD4667
S1131A9002B080BD80F00F40C0F00F4000F10F4055
S1131AA040F00F4080B586B000AF3A60FB1D021CC9
S1131AB01A70BB1D0A1C1A70BB1D1B78002B03D1A6
S1131AC02D4B00221A7053E0BB1D1B78022B03D14F
S1131AD0294B01221A704BE0BB1D1B78042B38D113
S1131AE0264B1B78DBB2012B33D13B683B613B694E
S1131AF09B883A1C0E3299B2402900D940231380A6
S1131B003B1C173300221A7012E03B1C17331A785F
S1131B103B6919683B1C17331B78CB181978184B91
S1131B2099543B1C17333A1C1732127801321A703D
S1131B303B1C17331B789BB23A1C0E3212889A4214
S1131B40E3D8104B3A1C173212781A70C046C046BC
S1131B500EE0BB1D1B78032B0AD1084B1B78DBB2AC
S1131B60012B05D1002002210022002303F086FD71
S1131B70C046BD4606B080BD0400002000F0FF1F33
S1131B80080000208800002080B582B000AF3A60D1
S1131B90FB1D021C1A70BB1D0A1C1A70074B1B7814
S1131BA0DBB2012B06D1BB1D1B78222B02D1044BC7
S1131BB001221A70C046BD4602B080BD0400002058
S1131BC000F0FF1F90B585B000AF041C081C111C69
S1131BD01A1CFB1D1C70BB1D18707B1D1970BB1CCF
S1131BE01A80BB1D1B78032B6BD1BB1C1B88002BDD
S1131BF009D1444B1A683B6A1A60424B1B791A1C80
S1131C007B6A1A8078E07B1D1B78022B57D83B1C1B
S1131C100F3300221A703B1C0E3301221A7020E08D
S1131C203B1C0F331A7837480821131C5B009B18A0
S1131C309B00C3185B181B88BA1C12889A4209D1EE
S1131C407B1D1B78022B12D83B1C0E337A1D127895
S1131C501A700CE03B1C0F333A1C0F32127801321D
S1131C601A703B1C0F331B78002BD9D000E0C04600
S1131C703B1C0F331A782349131C5B009B189B00F1
S1131C80CB180C331A683B1C0E331B789B00D318FB
S1131C901A683B6A1A603B1C0F331A781949131CE3
S1131CA05B009B189B00CB1810331A683B1C0E3347
S1131CB01B78D3181B781A1C7B6A1A801CE0C82373
S1131CC01BE0BB1D1B78072B14D8BB1D1A780E4BC9
S1131CD09200D2583B6A1A603B6A1B68002B01D100
S1131CE0CD230AE0BB1D1A78084B5200D25A7B6AF6
S1131CF01A8001E0CD2300E00023181CBD4605B086
S1131D0090BDC046F8720000C4720000B4720000B6
S1131D1080B582B000AF3A60FB1D021C1A70BB1D77
S1131D200A1C1A70BB1D1B78012B07D8BB1D1B781E
S1131D30054AD25C3B681A70002300E0CD23181CCE
S1131D40BD4602B080BDC0469C00002080B582B074
S1131D5000AFFB1D1870BB1D19707B1D1A70BB1DD5
S1131D601B78012B07D8BB1D1B78054A791D097800
S1131D70D154002300E0CD23181CBD4602B080BD21
S1131D809C00002080B584B000AF0A1CFB1D011C20
S1131D9019703B1D1A803B1C0F3300221A7011E08E
S1131DA03B1C0F331B780C4AD35C3A1D12889A42B1
S1131DB001D101230CE03B1C0F333A1C0F32127883
S1131DC001321A703B1C0F331B78012BE8D9002316
S1131DD0181CBD4604B080BD1873000080B584B0E3
S1131DE000AF0A1CFB1D011C1970BB1D1A703B1CA3
S1131DF00F3300221A7011E03B1C0F331B780C4A7E
S1131E00D35CBA1D12789A4201D101230CE03B1C29
S1131E100F333A1C0F32127801321A703B1C0F3305
S1131E201B78012BE8D90023181CBD4604B080BDE3
S1131E309C00002080B582B000AF021CFB1D1A700C
S1131E400023181CBD4602B080BDC04680B582B0D8
S1131E5000AF021CFB1D1A70024B181CBD4602B0D9
S1131E6080BDC046A472000080B582B000AF3A6065
S1131E70FB1D021C1A70BB1D0A1C1A70BB1D1B78AB
S1131E80012B0AD8BB1D1A78131CDB009B1A054AC8
S1131E909A183B681A60002300E0CD23181CBD4645
S1131EA002B080BDC0F0FF1F90B585B000AF3A60AE
S1131EB0FB1D021C1A70BB1D0A1C1A70BB1D1B786B
S1131EC0012B26D83B1C0F3300221A701AE0BB1DCD
S1131ED01A783B1C0F331C783B6819683B1C0F3382
S1131EE01B780833CB1818780C49131CDB009B1A99
S1131EF01B19021C5A543B1C0F333A1C0F32127824
S1131F0001321A703B1C0F331B78062BDFD90023D8
S1131F1000E0CD23181CBD4605B090BDC0F0FF1FE6
S1131F2080B582B000AF3A60FB1D021C1A70BB1D65
S1131F300A1C1A70BB1D1B78012B08D8BB1D1B780B
S1131F405A00054BD2183B681A60002300E0CD23E9
S1131F50181CBD4602B080BD9400002080B582B03C
S1131F6000AF3A60FB1D021C1A70BB1D0A1C1A70DC
S1131F70BB1D1B78012B08D8BB1D1B785A00054BD1
S1131F80D2183B681A60002300E0CD23181CBD461C
S1131F9002B080BD9800002080B584B000AF3A60E4
S1131FA0FB1D021C1A70BB1D0A1C1A70BB1D1B787A
S1131FB0012B22D83B1C0F3300221A7016E0BB1DE4
S1131FC018783B1C0F331A783B6819683B1C0F3395
S1131FD01B78CB1819780B4B40008218D1543B1C4A
S1131FE00F333A1C0F32127801321A703B1C0F3334
S1131FF01B78012BE3D9002300E0CD23181CBD4638
S113200004B080BD9400002080B584B000AF3A6075
S1132010FB1D021C1A70BB1D0A1C1A70BB1D1B7809
S1132020012B22D83B1C0F3300221A7016E0BB1D73
S113203018783B1C0F331A783B6819683B1C0F3324
S11320401B78CB1819780B4B40008218D1543B1CD9
S11320500F333A1C0F32127801321A703B1C0F33C3
S11320601B78012BE3D9002300E0CD23181CBD46C7
S113207004B080BD9800002080B500AF204A2049FC
S1132080204BCB588021490119431E4BD1501C4A87
S11320901B491D4BCB588021C90319431A4BD150FE
S11320A01A4B802292005A60184B802292009A6048
S11320B0164B80229200DA60154B16221A70144BCC
S11320C010225A70124B20229A70114B104A127827
S11320D0D2B240210A43D2B21A700C4B8022520071
S11320E01A600C4B0B4A526901210A435A61094B8D
S11320F0084A526801210A435A60BD4680BDC04661
S113210000700440381000003410000000C0044087
S113211000600740C0F00F4080B582B000AF021CE1
S1132120FB1D1A7000E0C046074BDB78DAB22023AF
S11321301340DBB2002BF6D0034BFA1D12785A7110
S1132140BD4602B080BDC0460060074080B582B085
S113215000AFFB1D00221A7000E0C046084BDB787C
S1132160DBB2DBB25BB2002BF7DA054AFB1D527916
S11321701A70FB1D1B78181CBD4602B080BDC046FA
S11321800060074080B582B000AF021CBB1D1A80FE
S1132190BB1D1B881B0A9BB2DBB2181CFFF7BCFFDC
S11321A0BB1D1B88DBB2181CFFF7B6FFBD4602B08F
S11321B080BDC04680B582B000AF021CFB1D1A7002
S11321C0324B324A1278D2B240218A43D2B21A70C8
S11321D0FB1D1B78002B10D12C4B2C4A1278D2B249
S11321E004218A43D2B21A70284B284A1278D2B2F8
S11321F008218A43D2B21A703DE0FB1D1B78012BE3
S113220010D1224B214A1278D2B204210A43D2B20D
S11322101A701E4B1D4A1278D2B208218A43D2B2D8
S11322201A7028E0FB1D1B78022B10D1174B174A9C
S11322301278D2B204218A43D2B21A70134B134AD1
S11322401278D2B208210A43D2B21A7013E0FB1DED
S11322501B78032B0FD10D4B0C4A1278D2B20421F8
S11322600A43D2B21A70094B084A1278D2B2082132
S11322700A43D2B21A70054B044A1278D2B24021F2
S11322800A43D2B21A70BD4602B080BD0060074056
S113229080B582B000AF021CFB1D1A701C4B1C4A97
S11322A01278D2B240218A43D2B21A70FB1D1B7835
S11322B0062B20D89A00174BD3181B689F46144B43
S11322C000229A7018E0124B10229A7014E0104BFE
S11322D020229A7010E00E4B21229A700CE00C4BD5
S11322E022229A7008E00A4B23229A7004E0084BD9
S11322F026229A7000E0C046054B054A1278D2B2F5
S113230040210A43D2B21A70BD4602B080BDC04615
S1132310006007401C73000080B582B000AF0A1C47
S1132320FB1D011C1970BB1D1A70FB1D1B78012BB2
S113233012D1BB1D1A780823134006D1114B114A40
S1132340926801210A439A6018E00E4B0D4A5268C4
S113235001210A435A6011E0BB1D1A780823134077
S113236006D1084B074A526801210A435A6005E026
S1132370044B044A926801210A439A60BD4602B0A4
S113238080BDC046C0F00F4080B500AF214A21494E
S1132390214BCB58C821890119431F4BD1501D4AE9
S11323A01C491E4BCB588021090419431B4BD150A7
S11323B01B4B802292005A611A4B802292005A6071
S11323C0174BA022D2009A61174B16221A70164B93
S11323D010225A70144B20229A70134B124A12780E
S11323E0D2B240210A43D2B21A70104B802252005A
S11323F05A630F4B0E4A5269802189010A435A617C
S11324000B4B0B4A5268802189010A435A60BD462E
S113241080BDC04600700440381000003410000035
S113242000C0044000D00440007007400090044005
S113243000F00F4080B582B000AF021CFB1D1A7083
S113244000E0C046074BDB78DAB220231340DBB24E
S1132450002BF6D0034BFA1D12785A71BD4602B018
S113246080BDC0460070074080B582B000AFFB1D40
S113247000221A7000E0C046084BDB78DBB2DBB206
S11324805BB2002BF7DA054AFB1D52791A70FB1D6B
S11324901B78181CBD4602B080BDC04600700740C2
S11324A080B582B000AF021CBB1D1A80BB1D1B8807
S11324B01B0A9BB2DBB2181CFFF7BCFFBB1D1B88B9
S11324C0DBB2181CFFF7B6FFBD4602B080BDC046A4
S11324D080B582B000AF021CFB1D1A70324B324A29
S11324E01278D2B240218A43D2B21A70FB1D1B78F3
S11324F0002B10D12C4B2C4A1278D2B204218A43DF
S1132500D2B21A70284B284A1278D2B208218A43D0
S1132510D2B21A703DE0FB1D1B78012B10D1224B67
S1132520214A1278D2B204210A43D2B21A701E4B45
S11325301D4A1278D2B208218A43D2B21A7028E016
S1132540FB1D1B78022B10D1174B174A1278D2B2FD
S113255004218A43D2B21A70134B134A1278D2B2AE
S113256008210A43D2B21A7013E0FB1D1B78032B17
S11325700FD10D4B0C4A1278D2B204210A43D2B2C5
S11325801A70094B084A1278D2B208210A43D2B20F
S11325901A70054B044A1278D2B240210A43D2B2CF
S11325A01A70BD4602B080BD0070074080B582B08D
S11325B000AF021CFB1D1A701C4B1C4A1278D2B2CD
S11325C040218A43D2B21A70FB1D1B78062B20D8F7
S11325D09A00174BD3181B689F46144B00229A701D
S11325E018E0124B10229A7014E0104B20229A70BB
S11325F010E00E4B21229A700CE00C4B22229A70B0
S113260008E00A4B23229A7004E0084B26229A70B1
S113261000E0C046054B054A1278D2B240210A4375
S1132620D2B21A70BD4602B080BDC04600700740E9
S11326303873000080B582B000AF0A1CFB1D011C7A
S11326401970BB1D1A70FB1D1B78012B14D1BB1D07
S11326501A780823134007D1134B134A9268802138
S113266089010A439A601BE00F4B0F4A526880218C
S113267089010A435A6013E0BB1D1A7808231340EA
S113268007D1094B084A5268802189010A435A60DC
S113269006E0054B044A9268802189010A439A6046
S11326A0BD4602B080BDC04600F00F4080B584B086
S11326B000AF78600023FB600023FB6002E0FB684E
S11326C00133FB60FA687B6803494B439A42F6D3B3
S11326D0BD4604B080BDC0467701000080B500AFA0
S11326E00C4A0C490C4BCB588021090519430A4B61
S11326F0D1500A4B4D229A60084B1022DA60074BE6
S113270000221A62054B054A526A08218A435A621A
S1132710BD4680BD007004403C10000000B0034082
S113272080B582B000AFBB1D00221A80FFF7D6FF30
S11327304E4B4E4A526A40210A435A624B4B4B4A13
S1132740526A80210A435A62C046484B5A6A80231F
S11327501340FAD1454B5A6A4023134007D0434BE8
S1132760DB6C99B2BB1DBA1D12888A181A803F4BC4
S11327709B6C99B2BB1DBA1D12888A181A803B4BF8
S11327805B6C99B2BB1DBA1D12888A181A80374B2C
S11327901B6C99B2BB1DBA1D12888A181A80334B60
S11327A0DB6B99B2BB1DBA1D12888A181A802F4B95
S11327B09B6B99B2BB1DBA1D12888A181A80BB1D67
S11327C0BA1D128852081A80BB1DBA1D12882849E6
S11327D00A431A80254BBA1D1288DA62BB1D0022F7
S11327E01A80224BDB6E99B2BB1DBA1D12888A185F
S11327F01A801E4B9B6E99B2BB1DBA1D12888A1893
S11328001A801A4B5B6E99B2BB1DBA1D12888A18C6
S11328101A80164B1B6E99B2BB1DBA1D12888A18FA
S11328201A80124BDB6D99B2BB1DBA1D12888A182F
S11328301A800E4B9B6D99B2BB1DBA1D12888A1863
S11328401A80BB1DBA1D128852081A80BB1DBA1DFE
S1132850128807490A431A80044BBA1D12881A6366
S11328600023181CBD4602B080BDC04600B0034022
S11328700080FFFF80B582B000AF021CFB1D1A7000
S1132880044BFA1D11781F220A401A60BD4602B09B
S113289080BDC04600B0034080B584B000AF021CC8
S11328A0FB1D1A700023FB60FB1D1B78181CFFF72F
S11328B0E1FF02E0064B1B68FB60FA6880231340CB
S11328C0F8D0034B1B699BB2181CBD4604B080BDF5
S11328D000B0034098B500AF084C094B1B68094889
S11328E0191C04F081F8031C6360044B00229A60F5
S11328F0024B07221A60BD4698BDC04610E000E0B6
S1132900D4F0FF1F006CDC0290B585B000AF786096
S11329107A68FF231340FB607A683D4B13401B0A1F
S1132920BB60BA68131C5B009B18DB001A1C394B94
S11329301A60394C374B1B683848191C04F054F89A
S1132940031C6360FB680A3B502B28D89A00344B65
S1132950D3181B689F46334B02221A6023E0314B85
S113296004221A601FE02F4B06221A601BE02D4B35
S113297008221A6017E02B4B0A221A6013E0294B35
S11329800C221A600FE0274B0E221A600BE0254B35
S113299010221A6007E0234B12221A6003E0214B35
S11329A006221A60C0467B68002B17DA1E4B0122F0
S11329B01A601E4B1D4A926804210A439A601C4BFC
S11329C01B4A9268802109010A439A60184B184AED
S11329D092688021C9000A439A6016E0124B0022D3
S11329E01A60124B114A526804210A435A60104B70
S11329F00F4A5268802109010A435A600C4B0C4A61
S1132A0052688021C9000A435A60BD4605B090BD92
S1132A1000FFFF00D4F0FF1F10E000E0006CDC02B8
S1132A2054730000D0F0FF1FA800002000F10F40F5
S1132A3040F00F4080B500AF214B214A5268082175
S1132A400A435A60FA235B00181C00F0ADF81C4BD3
S1132A501B4A926810210A439A60FA235B00181CEF
S1132A6000F0A2F8164B164A526820210A435A6015
S1132A70FA235B00181C00F097F8114B104A926877
S1132A8008210A439A60FA235B00181C00F08CF8B2
S1132A900B4B0B4A526810210A435A60FA235B001D
S1132AA0181C00F081F8064B054A926820210A435D
S1132AB09A60FA235B00181C00F076F8BD4680BDCE
S1132AC000F10F4080B500AF324B1B68012B5ED183
S1132AD0314B1B685A1C304B1A602F4B1B68032B5D
S1132AE055D92D4B00221A602C4B1B68052B4AD854
S1132AF09A002B4BD3181B689F462A4B294A5268CD
S1132B0008210A435A60254B1B685A1C234B1A6040
S1132B103DE0244B234A926810210A439A601F4BDC
S1132B201B685A1C1D4B1A6031E01E4B1D4A52682B
S1132B3020210A435A60194B1B685A1C174B1A6010
S1132B4025E0184B174A926808210A439A60134BF0
S1132B501B685A1C114B1A6019E0124B114A526837
S1132B6010210A435A600D4B1B685A1C0B4B1A6008
S1132B700DE00C4B0B4A926820210A439A60074BE4
S1132B8000221A6003E0054B00221A60C046BD46CD
S1132B9080BDC046A800002054040020B4000020DA
S1132BA09874000000F10F4080B582B000AF7860E7
S1132BB0054B00221A60C046034B1A687B689A4290
S1132BC0FAD3BD4602B080BDA000002080B584B019
S1132BD000AF021C3960FB1D1A703B1C0F3300222E
S1132BE01A70054B3A681A603B1C0F331B78181C8B
S1132BF0BD4604B080BDC046B800002090B587B083
S1132C0000AFB9607A603B603B1C0F33021C1A7042
S1132C10BB689B88DAB20C4B1A700B4B1A783C1CBD
S1132C2017343B1C0F3319787B68081C111C1A1CC1
S1132C30FFF71AF9031C23703B1C17331B78181C6D
S1132C40BD4607B090BDC046C000002090B587B017
S1132C5000AFB9607A603B603B1C0F33021C1A70F2
S1132C603B6800221A80BB689B88DAB20C4B1A704E
S1132C700B4B1A783C1C17343B1C0F3319783B1C44
S1132C800833081C111C1A1CFFF70EF9031C2370CF
S1132C903B1C17331B78181CBD4607B090BDC046BB
S1132CA0C000002080B584B000AFB9607A603B609A
S1132CB03B1C0F33021C1A703B6800221A80BB684D
S1132CC05B88DAB22A4B1A702A4B00221A70284BFE
S1132CD01B781A1C022313405A1E9341D9B2254B68
S1132CE001220A4052001978022081430A431A70D3
S1132CF01F4B1B781A1C022313405A1E9341D9B24E
S1132D001C4B01220A401978012081430A431A709E
S1132D10174B1A7801231340DAB2174B1A703B1C75
S1132D200F331B78181C00F0D7F8144B1B68002BCA
S1132D3018D00F4B1B781A1C0223134009D00F4BD9
S1132D401B683A1C0F321278101C2221002298476B
S1132D5008E00A4B1B683A1C0F321278101C212120
S1132D60002298470023181CBD4604B080BDC0460D
S1132D70BD000020C4000020BC000020B8000020DA
S1132D8080B584B000AFB9607A603B603B1C0F3300
S1132D90021C1A703B6800221A80BB685A88034BD5
S1132DA01A800023181CBD4604B080BDBE0000205C
S1132DB090B587B000AFB9607A603B603B1C0F33BD
S1132DC0021C1A703B1C173300221A703B68022243
S1132DD01A80BB689B88DAB2194B1A70BB685B888F
S1132DE0012B0FD1164B1A783C1C17343B1C0F33A4
S1132DF019787B68081C111C1A1CFFF791F8031C36
S1132E00237016E0BB685B88022B0FD10C4B1A7839
S1132E103C1C17343B1C0F3319787B68081C111CAD
S1132E201A1CFFF79BF8031C237002E03B68002286
S1132E301A803B1C17331B78181CBD4607B090BD85
S1132E40C000002090B587B000AFB9607A603B60E5
S1132E503B1C0F33021C1A703B1C173300221A70E0
S1132E603B6802221A80BB689B88DAB2194B1A703D
S1132E70BB685B88012B0FD1164B1A783C1C1734A6
S1132E803B1C0F3319787B68081C111C1A1CFFF7B4
S1132E9083F8031C237016E0BB685B88022B0FD1F8
S1132EA00C4B1A783C1C17343B1C0F3319787B6885
S1132EB0081C111C1A1CFFF7A7F8031C237002E05E
S1132EC03B6800221A803B1C17331B78181CBD4634
S1132ED007B090BDC000002080B582B000AF021CD6
S1132EE0FB1D1A70094B1A78094B1A71094B1A7891
S1132EF0074B1A72FB1D1A78054B101C03211A1C70
S1132F000A2300F037FCBD4602B080BDC00000209B
S1132F10D8F0FF1FC400002090B589B000AF7860DE
S1132F207B681B78181CFEF791FF031CBB613B1CDC
S1132F301F3300221A7014E03B1C1F331A78B9693E
S1132F40131C9B009B18CB1801331A787B685B78A1
S1132F509A420ED03B1C1F333A1C1F3212780132A6
S1132F601A70BB691B783A1C1F3212789A42E3D359
S1132F7000E0C0463B1C1F331A783B1C173337490B
S1132F80342042438A18D2781A707B681B7A002B4B
S1132F900ED13B1C1F331B78304934225A438A1804
S1132FA092780132D2B22D4934204343CB189A701F
S1132FB03B1C1F331A783B1C1633284934204243E8
S1132FC08A1892781A703A1C16323B1C17331278FE
S1132FD01B789A4225D03B1C1F331C783B1C1633AC
S1132FE01A7803231A40391C08311C48131C5B004F
S1132FF09B189B00342262439A1804238218D21827
S11330000B1C13CA13C33B1C083318783B1C08332E
S113301059783B1C08335A683B1C08331B8901F060
S113302067FC0F4B1B68002B15D03B1C1E3303227F
S11330301A707B681B7A002B03D03B1C1E330522BD
S11330401A70074B1B687A6810787A680832391C42
S11330501E3109789847BD4609B090BDD0000020C4
S1133060C800002090B58BB000AF78607B681B78F7
S1133070181CFEF7EBFE031C3B627B681A79597936
S113308009020A43997909040A43DB791B061343AD
S11330901A1C3B1C14331A607B685A7A9B7A1B02F5
S11330A013439AB23B1C14339A803B1C27330022EF
S11330B01A7014E03B1C27331A78396A131C9B00DE
S11330C09B18CB1801331A787B685B789A420ED030
S11330D03B1C27333A1C2732127801321A703B6AA0
S11330E01B783A1C273212789A42E3D300E0C04698
S11330F03B1C27331A783B1C1F3338493420424386
S11331008A18D2781A707B681B7A002B0ED13B1C6C
S113311027331B78314934225A438A189278013272
S1133120D2B22E4934204343CB189A703B1C273328
S11331301A783B1C1E332949342042438A1892785A
S11331401A703A1C1E323B1C1F3312781B789A42A9
S113315025D03B1C27331C783B1C1E331A780323D1
S11331601A40391C08311D48131C5B009B189B0036
S1133170342262439A1804238218D2180B1C13CAEF
S113318013C33B1C083318783B1C083359783B1C89
S113319008335A683B1C08331B8901F0A9FB104B08
S11331A01B68002B16D07B681B7A002B09D00C4BB4
S11331B01B687A6811787A680832081C05219847D8
S11331C008E0074B1B687A6811783A1C1432081C13
S11331D003219847BD460BB090BDC046D0000020E7
S11331E0C800002080B584B000AF78607B681A798D
S11331F0597909020A43997909040A43DB791B06C0
S113320013431A1C3B1C08331A607B685A7A9B7A56
S11332101B0213439AB23B1C08339A800E4B1B6863
S1133220002B16D07B681B7A002B09D00A4B1B6835
S11332307A6811787A680832081C0521984708E0F2
S1133240054B1B687A6811783A1C0832081C042163
S11332509847BD4604B080BDC800002090B58BB02F
S113326002AF3A60FB1D021C1A70BB1D0A1C1A70C7
S1133270FB1D1B78181CFEF7E9FD031CBB61BB1D7D
S11332801B78022B00D09BE03B1C1E3300221A70DB
S11332903B1C173300221A703B1C163300221A7091
S11332A03B1C1733BA6912781A703B1C1E333A1C44
S11332B0163212781A701AE03B1C1E331A78131C4B
S11332C09B009B18BA69D31801333B613B691A7898
S11332D03B699B78F91D081C111C1A1C03F01AFA8F
S11332E03B1C1E333A1C1E32127801321A703B1CEE
S11332F01E331A783B1C173319783B1C16331B7882
S1133300CB189A42D8DB3B1C1E333A1C1632127877
S11333101A7048E03B1C1E331A78131C9B009B1840
S1133320BA69D3180133FB60FB681978FB68DA7853
S11333301B791B0213439AB2FB689B78F8684478A4
S1133340F81D00940024019403F080F9FB685B7875
S1133350022B0DD0032B0AD1FB1D1978FB681A78B8
S1133360334B081C111C1A1C03F0DEFA01E000E0C8
S1133370C046FB681B7810221343DBB2DAB2FB6849
S11333809B78DB01DBB21343DBB2DBB2FA1D101C0A
S1133390191C002203F042FA3B1C1E333A1C1E3255
S11333A0127801321A703B1C1E331A783B1C1733F7
S11333B019783B1C16331B78CB189A42AADB28E0F9
S11333C0BB1D1B78002B24D13B1C1F3300221A7019
S11333D018E03B1C1F331B78164A34214B43D31887
S11333E000229A703B1C1F331B78124A34214B4332
S11333F0D3180022DA703B1C1F333A1C1F32127898
S113340001321A70BB691B783A1C1F3212789A4237
S1133410DFD3094B1B68002B07D0074B1B68FA1D31
S11334201078BA1D11783A689847BD4609B090BD26
S1133430192F0000D0000020C8000020B0B586B0CD
S113344000AFB9607A603B603B1C0F33021C1A70FA
S11334503B1C1733CD221A70BB681B781A1C6023DF
S11334601340202B00D085E03B1C173300221A7038
S1133470BB685B78232B00D978E09A004D4BD318B6
S11334801B689F463B6800221A808BE03B68002241
S11334901A8087E03C1C17343B1C0F331878B9683A
S11334A07A683B68FFF7CEFC031C23707AE03C1C6F
S11334B017343B1C0F331878B9687A683B68FFF7F8
S11334C077FC031C23706DE03B6802221A807B6842
S11334D01B6800221A707B681B685A1C7B681A6080
S11334E07B681B6800221A703C1C17343B1C0F338A
S11334F01878B9687A683B68FFF7A4FC031C23704A
S113350050E03C1C17343B1C0F331878B9687A68B8
S11335103B68FFF773FB031C237043E03C1C173428
S11335203B1C0F331878B9687A683B68FFF78EFB49
S1133530031C237036E03C1C17343B1C0F331878F3
S1133540B9687A683B68FFF7ADFB031C237029E078
S11335503C1C17343B1C0F331878B9687A683B68F5
S1133560FFF70EFC031C2370C0461BE03B680022DF
S11335701A8017E0BB681B781A1C60231340402B89
S113358010D10D4B1B68002B0CD00B4B1D683C1C41
S113359017343B1C0F331878B9687A683B68A8471E
S11335A0031C23703B1C17331B78181CBD4606B044
S11335B0B0BDC046B0740000CC00002090B587B008
S11335C000AFB9607A603B603B1C0F33021C1A7079
S11335D03B1C163300221A703B1C0F331B78181C3B
S11335E0FEF734FC031C3B613B691B780133DAB200
S11335F03C1C16343B1C0F3319783B1C28331B78B6
S1133600081C002102F0E6FF031C23703B1C163348
S11336101B78002B6CD13C1C16343B1C0F331978DF
S1133620374A384B081C111C1A1C00F0FBFF031C02
S113363023703B1C173300221A703BE03B1C1733EA
S113364018783B1C17331A783969131C9B009B1894
S1133650CB18013319782C4B34224243D1543B1CF0
S1133660173318783B1C17331A783969131C9B00DD
S11336709B18CB1802331A78234934234343CB18BD
S11336805A703B1C17331B781F4A34214B43D31801
S113369000229A703B1C17331B781B4A34214B437E
S11336A0D3180022DA703B1C17333A1C17321278F5
S11336B001321A703B691B783A1C173212789A420D
S11336C0BCD33C1C16343B1C0F331A783B68101CCB
S11336D0191CFFF77BFA031C23703B1C16331B7861
S11336E0002B05D1094BBA681A60094B7A681A6035
S11336F03B1C16331B78181CBD4607B090BDC04652
S11337005D3200003D340000D0000020C8000020DD
S1133710CC00002090B585B000AF021CFB1D1A70D0
S11337203B1C0F3300221A70104B00221A60104BFE
S113373000221A603C1C0F34FB1D1B78181C01F07E
S11337401DF8031C23703B1C0F331B78002B05D181
S11337503C1C0F3402F06CFF031C23703B1C0F3322
S11337601B78181CBD4605B090BDC046C80000209B
S1133770CC00002090B587B000AF3A601A1CFB1D46
S11337801870BB1D19703B1D1A803B1C1733002297
S11337901A70FB1D1B78181CFEF758FB031C3B61B9
S11337A03B1C163300221A7014E03B1C16331A78A3
S11337B03969131C9B009B18CB1801331B78BA1D65
S11337C012789A420ED03B1C16333A1C16321278E9
S11337D001321A703B691B783A1C163212789A42ED
S11337E0E3D300E0C0463B1C16331A783B1C0F336E
S11337F04F49342042438A18D2781A703B1C16333E
S11338001A783B1C0E334A49342042438A18927872
S11338101A703A1C0F323B1C0E3312781B78D31AE1
S1133820DBB2042B79D03B1C0D333A1C0F321178D8
S113383003220A401A703B1C163318783B1C0D33C4
S11338401A783B49131C5B009B189B0034224243AB
S11338509B18FA1DCB1812781A713B1C1633187872
S11338603B1C0D331A783249131C5B009B189B00D8
S1133870342242439B18BA1DCB1812785A713B1C50
S1133880163318783B1C0D331A782949131C5B0036
S11338909B189B00342242439B18CB1808333A6888
S11338A01A603B1C163318783B1C0D331A782049D8
S11338B0131C5B009B189B00342242439B183A1D47
S11338C0CB1812889A813B1C16331B783A1C0F3292
S11338D0391C0F31097801311170154934225343D1
S11338E03A1C0F32CB181278DA703A1C0F323B1C98
S11338F00E3312781B78D31ADBB2012B11D13C1C86
S11339001734FB1D1878BB1D19783A683B1D1B88BA
S113391000F0EEFF031C237003E03B1C1733C122AD
S11339201A703B1C17331B78181CBD4607B090BD9A
S1133930D000002090B587B000AFB9607A603B1C1E
S11339400F33021C1A703B1C173300221A700D4BE4
S1133950BA681A600C4B7A681A603C1C17343B1C1A
S11339600F331A78094B101C00211A1C02F0DCFFDB
S1133970031C23703B1C17331B78181CBD4607B06F
S113398090BDC046780100207C010020E939000088
S113399090B585B000AF021CFB1D1A700A4B0022C3
S11339A01A600A4B00221A603C1C0F34FB1D181CC1
S11339B0002102F0C9FF031C23703B1C0F331B784A
S11339C0181CBD4605B090BD780100207C01002084
S11339D080B582B000AF021CFB1D1A700023181CB6
S11339E0BD4602B080BDC046B0B588B002AF7860B5
S11339F03B1C163300221A703B1C1733CD221A705D
S1133A0000233B617A683B1C1633101C01211A1CED
S1133A1002F0C2FE7B689B78012B00D0A2E07B6899
S1133A201A79597909020A43997909040A43DB7915
S1133A301B0613436C4A101C191C082203F040F89F
S1133A40694B9A88684B9A80674B5A88664B5A80B0
S1133A50654BDA88644BDA80634B1B781A1C60234D
S1133A6013402ED1604B5B781A1C604B9200D358E4
S1133A70002B69D03B1C16331B78022B64D85A4B9D
S1133A805B781A1C3B1C16331B78181C5849131CF2
S1133A905B009B181B185B5C012B55D1524B5B7868
S1133AA01A1C524B9200D5587B6818783C1C17346A
S1133AB04D493A1C10323B1C0E33A847031C23709B
S1133AC042E0494BDA883B1C0E331A803B1C0E3310
S1133AD01B88202B2BD83B1C0E331B88002B13D0A8
S1133AE0414B1B78DBB25BB2002B0DDB414B3E4AF2
S1133AF003CA03C379683B1C0E331B883E4A081C67
S1133B00002101F0BBFD6CE03C4B1B68002B1BD07B
S1133B103A4B1D687B6818783C1C173432493A1CB0
S1133B2010323B1C0E33A847031C23700CE07B6847
S1133B3019782D4A3B1C1033381C0E300090081C99
S1133B40CD2100F05DF84CE07B6818783B1C1733FE
S1133B501978254A3B1C10333C1C0E34009400F0A9
S1133B604FF83EE03B1C16331B78042B05D17B68D1
S1133B701B78181C00F08CFA33E01B4B1B78DBB26B
S1133B805BB2002B2DDB7B68DB78002B29D11B4B30
S1133B901B68002B18D07B685A7A9B7A1B0213434C
S1133BA09BB208339AB23B1C0E331A80134B1D6828
S1133BB07B6818783C1C17340E493A1C10323B1CA5
S1133BC00E33A847031C23707B6818783B1C1733FB
S1133BD01978054A3B1C10333C1C0E34009400F049
S1133BE00FF8BD4606B0B0BD6C010020687500003A
S1133BF04075000080010020880100207C01002025
S1133C0080B584B000AFBA607B603B1C0F33021CEC
S1133C101A703B1C0E330A1C1A703B1C0E331B78A3
S1133C20CD2B07D13B1C0F33181C9021012202F02D
S1133C30F5FD22E0BB691A88BB68DB889A4203D988
S1133C40BB68DA88BB691A803B1C0F3319787B6820
S1133C501A68BB691B88081C002100F049FEBB6878
S1133C601B78DBB25BB2002B07DA3B1C0F33181C4A
S1133C7000210022002301F001FDC046BD4604B02E
S1133C8080BDC04690B58BB002AFB9607A603B602E
S1133C903B1C0F33021C1A700023BB613B1C1E33F8
S1133CA000221A703B1C153303221A703C1C1F346B
S1133CB03A1C0F323B1C1533101C01211A1C02F054
S1133CC06BFD031C2370BB681B781A1C0323134071
S1133CD04AD13C1C1F343A1C0F323B1C1433101CB9
S1133CE006211A1C02F058FD031C23703B1C1433DC
S1133CF01B781A1C534B1A80524B1A880323134007
S1133D009AB2504B1A804F4B1A884E4B1A803B1C68
S1133D100F331B783C1C1F343A1C183200923A1C97
S1133D2016320192181C022100220023FDF74AFFDB
S1133D30031C2370BB6907331B781A1C40231340F0
S1133D4007D0404B1B88012213439AB23D4B1A8083
S1133D5006E03C4B1B88012293439AB2394B1A80EC
S1133D603B6802221A8063E0BB681B781A1C032399
S1133D701340012B1AD1BB689A883B1C1D331A705F
S1133D803B1C15331B78012B09D13B1C1D331B78BD
S1133D90002B04D03B1C1F33CD221A7048E0294B62
S1133DA000221A803B6802221A8041E0BB681B781B
S1133DB01A1C03231340022B3AD13B1C15331B78E6
S1133DC0012B09D13B1C1E331B78002B04D03B1C58
S1133DD01F33CD221A702BE0BB689B88DAB23B1CE0
S1133DE01E3310210A431A703C1C1F34391C0F3136
S1133DF03B1C1E331A783B1C1333081C111C1A1C61
S1133E0002F0CAFC031C23703B1C13331B781A1CDE
S1133E100C4B1A800B4B1A88012313409AB2094B9E
S1133E201A80084B1A88074B1A803B6802221A80B2
S1133E307B68044A1A603B1C1F331B78181CBD4660
S1133E4009B090BD7401002090B587B000AFB9608F
S1133E507A603B603B1C0F33021C1A703B1C173307
S1133E60CD221A703B6800221A80BB685B781A1C4A
S1133E70022313405A103B1C15331A70BB681B787D
S1133E801A1C0323134000D081E03B1C15331B781C
S1133E90012B3FD1BB685B88012B03D0BB685B88D7
S1133EA0022B32D13C1C17343A1C0F323B1C123308
S1133EB0101C06211A1C02F06FFC031C23703B1C0F
S1133EC017331B78002B00D0B9E0BB685B88DBB2EA
S1133ED00122111C99400B1CDAB23B1C12331B78D3
S1133EE01343DAB23B1C12331A703B1C12331B7897
S1133EF03C1C17343A1C0F32101C06211A1C02F009
S1133F008DFC031C2370C04699E03B1C1733CD2263
S1133F101A7094E0BB685B88012B33D13C1C1734C6
S1133F203A1C0F323B1C1233101C06211A1C02F0DF
S1133F3033FC031C23703B1C17331B78002B00D06D
S1133F407DE0BB685B88DBB20122111C99400B1C2D
S1133F50DBB2DB43DBB23A1C123212781340DAB222
S1133F603B1C12331A703B1C12331B783C1C173455
S1133F703A1C0F32101C06211A1C02F04FFC031CC1
S1133F8023705CE03B1C1733CD221A7057E0BB68EA
S1133F901B781A1C03231340022B50D1BB689B8847
S1133FA0DAB23B1C11331A703B1C11331B781022FC
S1133FB01343DAB23C1C1734391C0F313B1C153344
S1133FC01B78081C111C1A1C02F028FC031C23700B
S1133FD03B1C15331B78002B01D0072300E008237A
S1133FE03A1C16321370BB685B78012B1CD13B1C46
S1133FF0113319783B1C14330F220A401A703B1CEE
S113400011331A783B1C1333D2091A703B1C143336
S11340101A783B1C13331B78101C191C01F0E8FAA6
S11340203B1C163308221A70084B1B683A1C0F32CB
S113403010783A1C163211783A1C113298473B1CFE
S113404017331B78181CBD4607B090BD78010020BB
S113405080B584B000AFB9607A603B603B1C0F331D
S1134060021C1A703B6800221A803B1C0F33181C78
S11340700121042202F0D2FBBB685B88DAB2034B55
S11340801A700023181CBD4604B080BD76010020C0
S113409080B582B000AF021CFB1D1A700C4B1B785C
S11340A0FA1D101C191C01F0E7FCFB1D181C012152
S11340B0012202F0B3FB064B1B78FA1D101C0321EE
S11340C01A1C02F0ABFB0023181CBD4602B080BDD5
S11340D07601002080B586B000AFB9607A603B609D
S11340E03B1C0F33021C1A703B6801221A803A1CD5
S11340F00F323B1C1733101C04211A1C02F04CFB1A
S11341003B1C17331B781A1C064B1A80054B1A8864
S1134110044B1A807B68034A1A600023181CBD46AE
S113412006B080BD7401002090B587B000AFB960BF
S11341307A603B603B1C0F33021C1A703B1C173324
S1134140CD221A703B6800221A803B1C17330422CC
S11341501A70BB685A883B1C14331A803B1C0F33FB
S11341601A783B1C14331B88101C191CFDF70AFE1B
S1134170031C002B3CD03B1C163300221A703B1C42
S113418014331B88002B03D13B1C163301221A70F5
S11341903C1C17343A1C0F323B1C16331B78101C82
S11341A001211A1C02F03AFB031C23703B1C14333C
S11341B01B88DBB23C1C17343A1C0F32101C042140
S11341C01A1C02F02BFB031C23700D4B1B683A1CBA
S11341D00F3211783A1C1432081C01219847084BFD
S11341E01B683A1C0F321278101C022100229847D7
S11341F03B1C17331B78181CBD4607B090BDC04646
S11342007801002090B587B000AFB9607A603B6058
S11342103B1C0F33021C1A70BB681B781A1C032347
S11342201340012B01D0042318E03B6801221A80BB
S1134230BB689B88DAB23C1C17343B1C0F331978DB
S1134240084B081C111C1A1CFDF762FD031C23708B
S11342507B68044A1A603B1C17331B78181CBD4644
S113426007B090BD7401002090B587B000AFB9606D
S11342707A603B603B1C0F33021C1A703B680022BF
S11342801A80BB681B781A1C03231340012B01D02E
S1134290042312E0BB689B88DAB2BB685B88DBB29C
S11342A03C1C1734391C0F310978081C111C1A1CCA
S11342B0FDF74CFD031C23700023181CBD4607B0FA
S11342C090BDC04690B587B000AFB9607A603B60DE
S11342D03B1C0F33021C1A703B6802221A803C1CE0
S11342E017343A1C0F323B1C1633101C05211A1CC0
S11342F002F052FA031C23703B1C16331B781A1C61
S1134300054B1A807B68044A1A603B1C17331B78E0
S1134310181CBD4607B090BD74010020B0B588B02C
S113432002AFB9607A603B603B1C0F33021C1A7009
S1134330BB685B881B0A9AB23B1C17331A703B1C80
S11343401433012252421A803B1C1333FF221A7089
S11343503B1C1433BA6892881A80BB685A883B1C89
S113436013331A703C1C12343B1C0F3318783B1C5B
S1134370173319783B1C13331A783B1C14331B88EE
S11343807D6800953D680195FDF71CFC031C2370B6
S11343903B1C12331B78181CBD4606B0B0BDC0468A
S11343A080B582B000AF78607A680C4B101C012194
S11343B01A1C02F0F1F97B68181C0121802202F01A
S11343C02DFA074B1B687A681278101C0A21002208
S11343D09847C046BD4602B080BDC046AC0100202F
S11343E0A801002080B584B000AF78607A683B1CD7
S11343F00F33101C01211A1C02F0CEF93B1C0F33A1
S11344001B78802B07D17A68084B1B78101C01217C
S11344101A1C02F003FA064B1B687A681278101C07
S11344200B2100229847BD4604B080BDAC0100209A
S1134430A801002080B582B000AF78607B685B780B
S1134440002B0DD17A687B68DB78DB01DBB21021AD
S11344500B43DBB2DBB2101C191C002202F0DEF9A4
S1134460C046BD4602B080BD80B584B000AF786060
S11344707B681A79597909020A43997909040A432C
S1134480DB791B0613431A783B1C0E331A803B1C42
S11344900E333A1C0E32128812021A807B681A7983
S11344A0597909020A43997909040A43DB791B06FD
S11344B0134301331B78191C3B1C0E333A1C0E3278
S11344C012880A431A807A683B1C0E331B88DBB2BD
S11344D0101C05211A1C02F0A1F9C046BD4604B007
S11344E080BDC046B0B586B002AF78603B1C0833CF
S11344F001229A703B1C083300221A703B1C0833BB
S1134500D97800220A4010210A43DA70197900226E
S11345100A401A713B1C083300225A7079683B1C0C
S113452008331A783B1C08339B783C1C0F34081C56
S1134530111C1A1C02F0EEF8031C237078683B1C53
S1134540083319783B1C0833DA781B791B021343B0
S11345509AB23B1C08339B783C1C083465783C1C9D
S11345600F3400950125019502F070F8031C2370A7
S11345703B1C083300229A7079683B1C08331A7874
S11345803B1C08339B78081C111C1A1C02F0C2F84F
S113459078683B1C083319783B1C0833DA781B799C
S11345A01B0213439AB23B1C08339B783C1C08340F
S11345B0647800940124019402F048F87B68181C84
S11345C00121022202F02AF97B68181C062101222B
S11345D002F024F97B68181C9021002202F01EF9D5
S11345E0054B1B687A681278101C0021002298473A
S11345F0BD4604B0B0BDC046A801002080B582B05D
S113460000AF7860064B1B687A6811787A680832C4
S1134610081C05219847C046BD4602B080BDC0466F
S1134620A801002090B587B000AFB9607A603B1C48
S11346300F33021C1A703B1C0F3319783C1C1734BF
S1134640BA687B68081C111C1A1CFFF773F9031C59
S11346502370424BBA681A603B1C17331B78002B3B
S113466075D13B1C0F331A783D4B101C10211A1CBA
S113467002F05AF9031C191C3B1C17333A1C17325D
S113468012780A431A703B1C0F331A78354B101CEE
S113469012211A1C02F048F9031C191C3B1C173385
S11346A03A1C173212780A431A703B1C0F331A78DB
S11346B02D4B101C14211A1C02F036F9031C191C72
S11346C03B1C17333A1C173212780A431A703B1CEE
S11346D00F331A78254B101C13211A1C02F024F9ED
S11346E0031C191C3B1C17333A1C173212780A435B
S11346F01A703B1C0F331A781D4B101C17211A1CFF
S113470002F012F9031C191C3B1C17333A1C173214
S113471012780A431A703B1C0F331A78154B101C7D
S113472016211A1C02F000F9031C191C3B1C173338
S11347303A1C173212780A431A703B1C0F33181CA8
S11347400121032202F06AF80B4B03221A703B1C6E
S113475017331B78181CBD4607B090BDA801002074
S1134760E544000069440000A1430000E543000063
S113477035440000FD450000AC01002090B585B033
S113478000AF021CFB1D1A703B1C0F3300221A7071
S1134790354B00221A60FB1D181C102102F0D4F8BE
S11347A0031C191C3B1C0F333A1C0F3212780A43AA
S11347B01A70FB1D181C122102F0C6F8031C191CE8
S11347C03B1C0F333A1C0F3212780A431A70FB1D3C
S11347D0181C142102F0B8F8031C191C3B1C0F33DD
S11347E03A1C0F3212780A431A70FB1D181C13214D
S11347F002F0AAF8031C191C3B1C0F333A1C0F329D
S113480012780A431A70FB1D181C172102F09CF839
S1134810031C191C3B1C0F333A1C0F3212780A4339
S11348201A70FB1D181C162102F08EF8031C191CAB
S11348303B1C0F333A1C0F3212780A431A703B1C8C
S11348400F331B78002B08D1FB1D1B783C1C0F3445
S1134850181CFFF79DF8031C23703B1C0F331B78B7
S1134860181CBD4605B090BDA801002080B584B0D9
S113487000AF021CFB1D1A70FA1D3B1C0F33101CE9
S113488001211A1C01F088FFFA1D3B1C0E33101C79
S113489006211A1C01F080FF3B1C0F331B78802B70
S11348A01ED13B1C0E331B781A1C0223134017D055
S11348B0FB1D1B78181CFDF7BDFA031C012B0FD13F
S11348C072B6FB1D181C01F00DF93B1C0F330022BE
S11348D01A70FB1D181C0121002201F09FFF62B613
S11348E03B1C0F331B78181CBD4604B080BDC0466A
S11348F090B585B000AF3A601A1CFB1D1870BB1D43
S113490019703B1D1A803B1C0F3300221A70FB1DCB
S11349101B783C1C0E34181CFFF7A8FF031C2370E3
S11349203B1C0E331B78802B0BD03B1D1B883C1C7F
S11349300F34F81DBA1D11783A6800F0E9FF031C22
S113494023703B1C0F331B78181CBD4605B090BD6B
S113495080B500AFBD4680BD80B500AF2D4A882329
S1134960BF21D1542B4A2B499423CB5CDBB20221C7
S11349700B43D9B29423D154264A98230021D1540D
S1134980244A80235B000021D154234A90239B00B6
S1134990101C191CFF2201F0CFFD204B1A68802344
S11349A0DB00101C191C002201F0C6FD1B4B1B6808
S11349B0802189005A181A4B1A601A4BFF221A7068
S11349C0144A14499423CB5CDBB202218B43D9B241
S11349D09423D1540F4A0F4986235B00CB5CDBB28E
S11349E040210B43D9B286235B00D154094A8C235E
S11349F0BF21D154074A84239F21D154054A054934
S1134A009423CB5CDBB220218B43D9B29423D154C1
S1134A10BD4680BD00200740B4010020B001002045
S1134A20F8030020E4F0FF1F80B584B000AFFB1D45
S1134A301870BB1D19707B1D1A703B1C0F33FF22AD
S1134A401A70FB1D1B78062B14D8FB1D1B789B00CA
S1134A50D9B23B1C0F337A1D12788A181A70BB1D09
S1134A601B78012B06D13B1C0F333A1C0F321278F2
S1134A7002321A703B1C0F331B78181CBD4604B05D
S1134A8080BDC04690B585B000AFFB1D1870BB1D3E
S1134A9019707B1D1A703C1C0F34FB1D1978BB1D4B
S1134AA01A787B1D1B78081C111C1A1CFFF7BCFF0D
S1134AB0031C23703B1C0F331B78FF2B12D03B1CB1
S1134AC00F331B785B08DBB21A1C0A49131CDB008A
S1134AD09B185B005A5A084B9A4203D13B1C0F3374
S1134AE0FF221A703B1C0F331B78181CBD4605B0FF
S1134AF090BDC046B4010020FFFF000090B585B012
S1134B0000AF786039603B689A79D97909020A4321
S1134B10197A09040A435B7A1B0613431A1C3B687F
S1134B20197B5B7B1B020B439BB2D318BB603B1C02
S1134B300E3300221A803B689A7ADB7A1B021343F5
S1134B409BB21A1C3B68197B5B7B1B020B439BB219
S1134B50D21A3B6819785B781B020B439BB29A42CA
S1134B6008DD3A1C0E323B6819785B781B020B4354
S1134B7013800FE03B689A7ADB7A1B02134399B2E5
S1134B803B681A7B5B7B1B0213439AB23B1C0E33BC
S1134B908A1A1A807B683A1C0E3211789C7800209D
S1134BA02040014399705278D878002101400A438B
S1134BB0DA70BA687B68FF2111401C79002020401C
S1134BC001431971100AFF2101405C790020204043
S1134BD001435971100CFF2101409C7900202040B1
S1134BE001439971120ED879002101400A43DA7108
S1134BF0BD4605B090BDC04680B582B000AF0A1C6A
S1134C00FB1D011C1970BB1D1A70494A80235B00EF
S1134C100021D154474BFA1D12781A70464A90234A
S1134C209B00101C191CFF2201F086FC434B444AD4
S1134C301A60424B1A688023DB00101C191C0022E6
S1134C4001F07AFC3F4BFF221A70394A3849862317
S1134C505B00CB5CDBB240210B43D9B286235B0003
S1134C60D154BB1D1B78002B07D0374B364A126832
S1134C70802109060A431A6005E0334B324A126860
S1134C80520052081A602A4A2C4B1B681B0ADBB2DA
S1134C9001218B43D9B29C23D154254A274B1B684D
S1134CA01B0CD9B2B023D154214A244B1B681B0ED0
S1134CB0D9B2B423D154214B1B68802189005A18DE
S1134CC0224B1A601A4A84235B001021D154184ADB
S1134CD094230121D154164A8023BF21D154144A6C
S1134CE0134980235B00CB5CD9B27F230B40D9B23C
S1134CF080235B00D1540E4A0D498423CB5CDBB284
S1134D0001210B43D9B28423D154094A084984238D
S1134D10CB5CDBB210210B43D9B28423D154044BB6
S1134D2084221A770023181CBD4602B080BDC046F9
S1134D3000200740F4030020B4010020B00100204B
S1134D4000060020E4F0FF1F00700440F803002078
S1134D5080B500AF174A174986235B00CB5CDBB2F2
S1134D6040218B43D9B286235B00D154114A80235E
S1134D70BF21D1540F4A0F498423CB5CDBB20121FC
S1134D808B43D9B28423D1540A4A0A499423CB5C75
S1134D90DBB201218B43D9B29423D154054B054A8C
S1134DA0127FD1B27B220A40D2B21A770023181C98
S1134DB0BD4680BD0020074090B589B000AF396082
S1134DC0FB1D011C1970BB1D1A703B1C1F333A6874
S1134DD012781A703B1C1E333A6892781A703B1C86
S1134DE00C33C64A03CA03C33B68DA781B791B0237
S1134DF013439AB280239B009A420AD93B68D9781C
S1134E0000220A40DA70197900220A4002210A437A
S1134E101A713C1C1D343B1C1F331A783B1C1E3377
S1134E201B78101C191C0022FFF7FEFD031C2370C5
S1134E303B1C1C333A1C1D32127852081A703B1C5E
S1134E401D331B78FF2B13D03B1C1C331A78AC4941
S1134E50131CDB009B185B005A5AAA4B9A4207D1D9
S1134E603B685B78032B03D83B689B78012B01D903
S1134E7095233EE13B1C1C331A78131CDB009B1862
S1134E805B009F4A9B18BB61BB69DB7BFF2B02D194
S1134E90BB690022DA733B68DA781B791B0213437F
S1134EA09AB2BB69FF2111401C78002020400143C5
S1134EB01970120A92B25878002101400A435A70BC
S1134EC0BB69BA1D12789A73BB69DA7B012313405C
S1134ED0DAB2BB69DA73BB69DB7BDAB23B1C1E3323
S1134EE01B785B00D9B23B1C1F331B789B00DBB2E1
S1134EF00B43DBB21343DBB2DAB2BB69DA73824B26
S1134F001A68BB69FF2111409C78002020400143AE
S1134F109970100AFF210140DC78002020400143F1
S1134F20D970100CFF2101401C790020204001435E
S1134F301971120E5879002101400A435A713B68D5
S1134F405A78BB695A74BB693A1C1E3212781A74B7
S1134F506E4B1A68BB69DB7BDB00D3187B613B6853
S1134F60DA781B791B0213439AB27B69FF21114043
S1134F709C780020204001439970120A92B2D8789C
S1134F80002101400A43DA705F4B1A687B69FF21F4
S1134F9011401C790020204001431971100AFF219F
S1134FA001405C790020204001435971100CFF211D
S1134FB001409C790020204001439971120ED87958
S1134FC0002101400A43DA717B6908221A704F4BB1
S1134FD01A68BB69DB7B01214B40DBB2DB00D318D1
S1134FE07B613B68DA781B791B0213439AB27B69B5
S1134FF0FF2111409C780020204001439970120A3F
S113500092B2D878002101400A43DA703E4B1A6804
S11350107B69FF2111401C79002020400143197154
S1135020100AFF2101405C7900202040014359719E
S1135030100CFF2101409C7900202040014399710C
S1135040120ED879002101400A43DA717B694822A3
S11350501A703B68DA781B791B0213439BB21A1C43
S1135060294B1B68D218284B1A603B1C1E331B7833
S1135070002B0ED1254B1A68BB69DB7BDB00D318F0
S11350807B617B691B78802252421343DAB27B69CD
S11350901A703B1C1E331A783B1C1E3319783B1CB8
S11350A00C338900C9583B685B78012B01D001237C
S11350B000E0002319433B1C0C339200D1503B1CED
S11350C01F331B789B00124A9B183A1C1F3212781C
S11350D092000F4812181278D1B23A1C1E3210787E
S11350E03A1C0C3280008258D2B20A43D2B21A70EF
S11350F00023181CBD4609B090BDC0469C75000035
S1135100B4010020FFFF0000F8030020B0010020DC
S1135110C020074090B587B000AF7860FB1C1970C1
S1135120BB1C1A703B1C1733C4221A703C1C163467
S1135130FB1C1A78BB1C1B78101C191C0022FFF7DF
S1135140A1FC031C23703B1C15333A1C1632127845
S113515052081A703B1C16331B78FF2B37D03B1CAC
S113516015331A78131CDB009B185B001B4A9B1831
S11351703B611B4B1A683B69DB7BDB00D318FB608C
S1135180174B1A683B69DB7B01214B40DBB2DB0028
S1135190D318BB60FB681A787F231340DAB2FB682C
S11351A01A70BB681A787F231340DAB2BB681A708E
S11351B03B699A7A012149420A439A72DA7A0121B7
S11351C049420A43DA723B1C173300221A703B1C13
S11351D017331B78181CBD4607B090BDB4010020DE
S11351E0B001002090B585B000AFFB1D1870BB1D49
S11351F019707B1D1A703C1C0F34BB1D1A787B1D63
S11352001B78101C191C0022FFF73CFC031C2370A4
S11352103B1C0E333A1C0F32127852081A703B1C96
S11352200F331B78FF2B01D196233EE0F91DBB1DE4
S11352301A787B1D1B78081C111C1A1CFFF76AFFC7
S11352401C4B19683B1C0E331A781B48131CDB00DB
S11352509B185B001B5ACA1A164B1A60BB1D1B789D
S11352609B00164A9B1800221A703B1C0E331A78B6
S11352701149131CDB009B185B00012252425A5255
S11352803B1C0E3319780C4A0B1CDB005B185B00CB
S1135290D11848880124644220434880D3189A884E
S11352A0012149420A439A800023181CBD4605B0D7
S11352B090BDC046F8030020B4010020C020074080
S11352C090B585B000AF7860FB1C1970BB1C1A70D8
S11352D03C1C0F34FB1C1A78BB1C1B78101C191CBB
S11352E00022FFF7CFFB031C23703B1C0F331B78FA
S11352F05B08DBB21A1C131CDB009B185B00164A0C
S11353009B18BB603B1C0F33BA68D27B1A703B1CE2
S11353100F331B78FF2B1BD07968FB1C1A78BB1C3E
S11353201B78081C111C1A1CFFF7F4FE0B4B1A689F
S11353303B1C0F331878094B1B68391C0F31097853
S1135340C900CB5C7C2149420B43D9B2C3009954B8
S1135350C046BD4605B090BDB4010020B001002098
S113536090B587B000AF7860FB1C1970BB1C1A7035
S11353703C1C1734FB1C1A78BB1C1B78101C191C12
S11353800022FFF77FFB031C23703B1C17331B78A1
S11353905B08DBB21A1C131CDB009B185B00354A4C
S11353A09B183B613B1C17333A69D27B1A703B1C38
S11353B017331B78FF2B58D0FB1C1B789B002E4AFD
S11353C09B18FB60FB1C1B78002B23D03B695B7C88
S11353D0012B01D0012300E000233A1C0B3213708F
S11353E0BB1C1B78012B01D1142300E018233A1CA9
S11353F00B3211781A1C0B1C1343DAB23B1C0B330F
S11354001A70FB681A783B1C0B331B781343DAB20F
S1135410FB681A70FB681A7802218A431A70174BCA
S11354201A683B1C17331878144B1B68391C173146
S11354300978C900C95C7B230B40D9B2C3009954D5
S11354400E4B1B683A1C17321278D2000021D1543B
S1135450BB1C1B78002B08D17A68FB1C1B78101C22
S1135460191C0022002300F009F9C046BD4607B00C
S113547090BDC046B4010020C0200740B001002008
S113548090B589B000AFF8607A603B1C0B330A1CFE
S11354901A703C1C1F343B1C0B331B78181C002156
S11354A00022FFF7EFFA031C23703B1C1F331B7809
S11354B05B08DBB21A1C131CDB009B185B00144A4C
S11354C09B18BB613B1C1F33BA69D27B1A70114B0A
S11354D01A683B1C1F331B78DB00D1180979D018DC
S11354E0407900020143D018807900040143D318A5
S11354F0DB791B060B437B617A687B69101C191CE2
S1135500082201F0DDFAC046BD4609B090BDC04690
S1135510B4010020B001002090B585B000AF7860E0
S1135520FB1C1970BB1C1A703B1C0F3305221A702C
S11355303C1C0E34FB1C1A78BB1C1B78101C191C59
S11355400022FFF79FFA031C23703B1C0E331B78C9
S1135550FF2B41D0FB1C1B789B0023495A183B1C92
S11355600D3312781A703B1C0F3300221A703B1C47
S11355700D331A780C23134004D13B1C0F3305223E
S11355801A7029E03B1C0D331A780223134004D00F
S11355903B1C0F3301221A701EE0144B1B683A1C8B
S11355A00E321278D200D35C1B06DB0FDBB2012B68
S11355B00ED00E4B1B683A1C0E32127801214A4061
S11355C0D2B2D200D35C1B06DB0FDBB2012B03D1BA
S11355D03B1C0F3303221A703B1C0F331B78181C1F
S11355E0BD4605B090BDC046C0200740B0010020B4
S11355F090B587B000AF0A1CFB1D011C1970BB1DC0
S11356001A703C1C1734FB1D1A78BB1D1B78101C28
S1135610191C0022FFF736FA031C23703B1C1733B6
S11356201B785B08DBB21A1C131CDB009B185B00A5
S11356300F4A9B183B613B1C17333A69D27B1A70A3
S11356403B1C17331B78FF2B0DD0FB1D1B789B00D5
S1135650084A9B18FB60084B1B683A1C17321278E7
S1135660D2000021D154C046BD4607B090BDC0460B
S1135670B4010020C0200740B001002090B589B0DB
S113568000AFF8607A603B603B1C0B330A1C1A7055
S11356903B1C1F3394221A703C1C1E343B1C0B33DE
S11356A01B78181C00210022FFF7ECF9031C23705F
S11356B03B1C1E331B785B08DBB21A1C131CDB007B
S11356C09B185B008F4A9B18BB613B1C1E33BA6955
S11356D0D27B1A703B1C1E331B78FF2B00D10AE1CE
S11356E0894B1A683B1C1E331B7801214B40DBB2EB
S11356F0DB00D3187B6100233B61BB691A785B78BC
S11357001B0213439AB2814B9A4200D1F3E07B69A6
S11357101B787F229343DBB2002B00D0EBE03B6885
S1135720002B56D1784B1A683B1C1E331B78DB00C8
S1135730D3183B61BB691A785B781B0213439AB296
S11357403B69FF2111409C7800202040014399705F
S1135750120A92B2D878002101400A43DA70BB6978
S11357609A78D97809020A43197909040A435B79BA
S11357701B0613431A1C3B69FF2111401C790020AE
S1135780204001431971100AFF2101405C79002077
S1135790204001435971100CFF2101409C790020E5
S11357A0204001439971120ED879002101400A4327
S11357B0DA713B691B785B06DB0FDBB29B01DBB262
S11357C0782252421343DBB2DAB23B691A700023E7
S11357D094E03B689AB2BB69FF2111409C7A002097
S11357E0204001439972120A92B2D87A00210140F2
S11357F00A43DA72BB693A1D127898790021014094
S11358000A439A717A1D1278D879002101400A431B
S1135810DA71BA1D1278187A002101400A431A720B
S1135820FA1D1278587A002101400A435A72BB6962
S11358301A785B781B0213439BB21A1C3B689A428A
S113584006D2BB691A785B781B0213439BB23B6098
S1135850BB69197B00220A401A73597B00220A4053
S11358605A73294B1A683B1C1E331B78DB00D31870
S11358703B613B689AB23B69FF2111409C78002050
S1135880204001439970120A92B2D8780021014055
S11358900A43DA707A683B69FF2111401C790020C1
S11358A0204001431971100AFF2101405C79002056
S11358B0204001435971100CFF2101409C790020C4
S11358C0204001439971120ED879002101400A4306
S11358D0DA713B691B785B06DB0FDBB29B01DBB241
S11358E0782252421343DBB2DAB23B691A703B1C92
S11358F01F3300221A703B1C1F331B78181CBD4633
S113590009B090BDB4010020B0010020FFFF0000E9
S113591090B589B000AFF8607A603B603B1C0B33F4
S11359200A1C1A703B1C1F3393221A703C1C1E3431
S11359303B1C0B331B78181C01210022FFF7A2F833
S1135940031C23703B1C1E331B785B08DBB21A1C40
S1135950131CDB009B185B00444A9B18BB613B1C77
S11359601E331B78FF2B01D193237AE03B1C1E339B
S1135970BA69D27B1A703E4B1A683B1C1E331B78E3
S1135980DB00D3187B617B691B787F229343DBB2F6
S1135990002B63D13B1C0B331B789B00354A9B18AF
S11359A01B78DBB21A1C0223134057D13B689AB20E
S11359B0BB69FF2111409C7A002020400143997269
S11359C0120A92B2D87A002101400A43DA72BB6902
S11359D03A1D12789879002101400A439A717A1D80
S11359E01278D879002101400A43DA71BA1D12787D
S11359F0187A002101400A431A72FA1D1278587A63
S1135A00002101400A435A72BB69197B00220A40F3
S1135A101A73597B00220A405A737A69BB69101CB5
S1135A20191CFFF76BF83B1C0B331B78002B03D1BD
S1135A307B69C8221A700DE07B691B785B06DB0F5B
S1135A40DBB29B01DBB2782252421343DBB2DAB2FF
S1135A507B691A703B1C1F3300221A703B1C1F33D6
S1135A601B78181CBD4609B090BDC046B401002087
S1135A70B0010020C020074080B582B000AF78603C
S1135A800A1CFB1C1A70074AF91C98230978D15484
S1135A90054B181C0121012200F0C0FEC046BD4682
S1135AA002B080BD00200740F403002080B582B01E
S1135AB000AF7860094A94230021D154074A862311
S1135AC05B008021D154064B181C0121FF2200F0F9
S1135AD0A5FEC046BD4602B080BDC04600200740BA
S1135AE0F403002080B584B000AF78602F4A2F49BA
S1135AF080235B00CB5CD9B27F230B40D9B28023D7
S1135B005B00D154294A294986235B00CB5CDBB274
S1135B1020218B43D9B286235B00D154234A2349E5
S1135B208023CB5CDBB220210B43D9B28023D15438
S1135B301E4A1E498423CB5CDBB220218B43D9B29D
S1135B408423D154194A19499423CB5CDBB2202114
S1135B508B43D9B29423D154144A14499423CB5C73
S1135B60DBB204210B43D9B29423D1543B1C0E3332
S1135B700F4A1A803B1C0E333A1C0E321288013A2B
S1135B801A80FAF76FFE3B1C0E331B88002BF1D1F1
S1135B90064A06499423CB5CDBB204218B43D9B279
S1135BA09423D154C046BD4604B080BD00200740B4
S1135BB0204E000090B589B000AF021C3960FB1D77
S1135BC01A703B1C1F3300221A700023BB61002390
S1135BD07B6100233B61FB1D1A78042313409A1058
S1135BE03B1C0F331A70FB1D1A7808231340DB107B
S1135BF0DAB23B68DA703B6859783B68DA783C1C67
S1135C001F343B1C0F331B78081C111C1A1CFEF795
S1135C100BFF031C2370A94B1A683B1C1F331B7812
S1135C20DB00D318BB61A54B1A683B1C1F331B78E0
S1135C3001214B40DBB2DB00D3187B613B1C1F33DB
S1135C401B785B08DBB21A1C131CDB009B185B007F
S1135C509B4A9B183B61BB691A79597909020A432B
S1135C60997909040A43DB791B0613431A1C3B6820
S1135C70FF2111401C790020204001431971100AB2
S1135C80FF2101405C790020204001435971100C30
S1135C90FF2101409C790020204001439971120E9C
S1135CA0D879002101400A43DA71BB699A78DB781C
S1135CB01B0213439AB23B68FF2111405C7A002017
S1135CC0204001435972120A92B2987A002101408D
S1135CD00A439A723B69DA7B3B1C1F3301214A4019
S1135CE01A703B693A1C1F321278DA73BB691B784D
S1135CF05B06DB0FDBB201225340DBB29B01DAB25D
S1135D007B691A703B68DB78012B00D0B7E03B68F5
S1135D105B78002B16D16B4B1B78002B12D1694B8F
S1135D20FF221A703B68181C00210022FFF7F2F9C9
S1135D307B6900221A703B68181C00210022002392
S1135D40FFF79CFC5F4B1B78012B04D03B685B780E
S1135D50002B00D138E23B691A7B5B7B1B021343A7
S1135D609AB23B68597A9B7A1B020B439BB2D318B5
S1135D709AB23B69FF2111401C7B00202040014363
S1135D801973120A92B2587B002101400A435A73D4
S1135D903B699A7ADB7A1B0213439AB23B69197BFB
S1135DA05B7B1B020B439BB29A4213D83B685A7A23
S1135DB09B7A1B0213439BB2DBB21A1C3B69197812
S1135DC05B781B020B439BB29A4218D13B699B7BC5
S1135DD0012B14D17A693B69101C191CFEF78EFE45
S1135DE07B691B785B06DB0FDBB29B01DBB278229D
S1135DF052421343DBB2DAB27B691A70ECE13B69BD
S1135E009A79D97909020A43197A09040A435B7A0F
S1135E101B0613431A1C3B68FF2111401C79002008
S1135E20204001431971100AFF2101405C790020D0
S1135E30204001435971100CFF2101409C7900203E
S1135E40204001439971120ED879002101400A4380
S1135E50DA713B691A7B5B7B1B0213439AB23B6882
S1135E60FF2111405C7A0020204001435972120A3C
S1135E7092B2987A002101400A439A72A4E13B68E5
S1135E805B78002B37D1BB691A783C231340DBB213
S1135E90342B19D13B6801229A703B681A795979DD
S1135EA009020A43997909040A43DB791B0613435F
S1135EB01B78DB09DAB2034B1A701CE0B001002036
S1135EC0B4010020E4F0FF1FC54B1B78012B12D155
S1135ED0C34BFF221A703B68181C00210122FFF7F4
S1135EE019F97B6900221A703B68181C00210022F2
S1135EF00023FFF7C3FB3B699A7ADB7A1B02134347
S1135F009AB2B84B9A4200D15EE13A1C0C323B681B
S1135F10597A9B7A1B020B4313803B691A7B5B7B88
S1135F201B0213439AB23B1C0C331B88D3189AB23E
S1135F303B69FF2111401C7B002020400143197361
S1135F40120A92B2587B002101400A435A733B69FA
S1135F501A785B781B0213439BB23A1C0C321288EA
S1135F609A420DD13B699A7ADB7A1B0213439AB2A7
S1135F703B69197B5B7B1B020B439BB29A4222D881
S1135F803B699A7ADB7A1B0213439BB2002B00D144
S1135F90D0E03B699A7ADB7A1B0213439AB23B69DD
S1135FA019785B781B020B439BB2101C191C00F080
S1135FB05FFD0B1C9BB2002B00D0BBE03B699B7BBD
S1135FC0012B00D0B6E03B699A7ADB7A1B021343BB
S1135FD09BB21A1C3B69197B5B7B1B020B439BB274
S1135FE0D21A3B6919785B781B020B439BB29A4225
S1135FF006DD3B691A785B781B0213439BB20DE004
S11360003B699A7ADB7A1B0213439AB23B69197B88
S11360105B7B1B020B439BB2D31A9BB23A1C0A3222
S113602013803B1C0A331B88002B33D13B699A78BD
S1136030D97809020A43197909040A435B791B06D2
S113604013431A1C7B69FF2111401C790020204056
S113605001431971100AFF2101405C79002020409E
S113606001435971100CFF2101409C79002020400C
S113607001439971120ED879002101400A43DA7163
S11360807B69997800220A409A70D97800220A40E4
S1136090DA7040E03B699A79D97909020A43197A9E
S11360A009040A435B7A1B0613431A1C3B69197BD8
S11360B05B7B1B020B439BB2D3181A1C7B69FF2129
S11360C011401C790020204001431971100AFF215E
S11360D001405C790020204001435971100CFF21DC
S11360E001409C790020204001439971120ED87917
S11360F0002101400A43DA717B693A1C0A321178A3
S11361009C7800202040014399705278D87800216F
S113611001400A43DA707B691B785B06DB0FDBB254
S11361209B01DBB2782252421343DBB2DAB27B69C1
S11361301A7051E03B699A79D97909020A43197AAC
S113614009040A435B7A1B0613431A1C3B68FF21AC
S113615011401C790020204001431971100AFF21CD
S113616001405C790020204001435971100CFF214B
S113617001409C790020204001439971120ED87986
S1136180002101400A43DA713B691A7B5B7B1B02E5
S113619013439AB23B68FF2111405C7A00202040EF
S11361A001435972120A92B2987A002101400A43BB
S11361B09A723B699A7A012149420A439A72DA7ABD
S11361C0012149420A43DA723B685A783B68101C41
S11361D0191C00F0DDFBC046BD4609B090BDC046A9
S11361E0E4F0FF1FFFFF000080B588B000AFCF4987
S11361F03B1C1F3380228A5C1A70CC493B1C1E3323
S113620084228A5C1A703B1C1D333A1C1F32391CD1
S11362101E31127809780A401A70C4493B1C1C3399
S113622090228A5C1A70FB1DFF221A70C04B1A78E8
S11362303B1C08331A703B1C083300229A703B1C29
S1136240083300225A603B1C08339968B94A0A4053
S11362509A603B1C08330022DA703B1C083300228E
S11362601A723B1C0833FF225A70B14AFB1D101CE2
S113627001211A1C00F090FAAC4A86235B00D35C1F
S1136280DBB21A1C012313401BD0FB1D1B78802B8F
S113629017D1A64AA54980235B00CB5CD9B27F23E2
S11362A00B40D9B280235B00D154A04A9F49862376
S11362B05B00CB5CDBB220218B43D9B286235B002D
S11362C0D1543B1C1D331A780423134031D0974A10
S11362D0A423D35CDAB23B1C1A331A803B1C183358
S11362E008221A80914AA023D35CDAB23B1C1633ED
S11362F01A808E4A80230421D1543B1C1A331A88F5
S11363003B1C18331B88111C99400B1C9AB23B1C74
S113631016331B8813439BB29AB23B1D1A803B1C55
S113632008333A1D5A603B1C08331220191C00F034
S11363302FFB3B1C1D331A780123134016D07B4AD4
S113634080230121D154FEF707FB3B1C08331020A6
S1136350191C00F01DFB754A74499423CB5CDBB215
S113636020218B43D9B29423D154DCE03B1C1D3350
S11363701A78082313401ED06C4A80230821D15474
S11363803B1C1C331B781B09DAB23B1C08335A70C4
S11363903B1C1C331A783B1C0833101C191CFFF7D8
S11363A009FC624A61499423CB5CDBB220218B4314
S11363B0D9B29423D1543B1C1D331A7802231340C1
S11363C02ED05A4A80230221D15458493B1C1F33F2
S11363D088228A5C1A7055493B1C1E338C228A5CC5
S11363E01A703B1C1F333A1C1E321B781278134060
S11363F0DAB23B1C08331A723B1C08331620191CF2
S113640000F0C6FA494A8823BF21D154474A474974
S11364109423CB5CDBB220218B43D9B29423D15497
S11364203B1C1D331A781023134030D03F4A80237D
S11364302021D1543D4A80231021D1543B1C0833E0
S11364401420191C00F0A4FA384A384986235B004A
S1136450CB5CDBB220210B43D9B286235B00D15441
S1136460324A324980235B00CB5CDBB28021494253
S11364700B43D9B280235B00D1542C4A2B4984238B
S1136480CB5CDBB220210B43D9B28423D1543B1C17
S11364901D331A782023134013D0244A802320214B
S11364A0D1543B1C08331320191C00F071FA1F4A05
S11364B01E498423CB5CDBB220218B43D9B28423D5
S11364C0D1543B1C1D331B785BB2002B2BDA3B1CD5
S11364D00833FF225A703A1C0832FB1C101C10218E
S11364E01A1C00F059F9FB1C1B78012B07D13B1C2B
S11364F0083300225A703B1C08330122DA700B4A1D
S113650080238021D1543B1C08331720191C00F030
S11365103FFA064A05499423CB5CDBB220218B4326
S1136520D9B29423D154BD4608B080BD00200740A1
S1136530F4030020FF0000FF80B584B000AFF860D2
S1136540B960FB1D1A70FB1D1A78F968BB68081C3A
S1136550111C1A1C00F0BDFAC046BD4604B080BD33
S113656080B582B000AFFB1D00221A70154B1A785B
S1136570154B1A70FB1D00221A7009E0FB1D1B78D5
S1136580124AFF21D154FB1DFA1D127801321A70F0
S1136590FB1D1B78062BF1D9FB1D00221A7009E0A4
S11365A0FB1D1B780A4A0521D154FB1DFA1D1278E4
S11365B001321A70FB1D1B78062BF1D9BD4602B0BF
S11365C080BDC0460C0400200B040020FC03002006
S11365D00404002080B582B000AF3960111C1A1C7D
S11365E0FB1D1870BB1D19707B1D1A70BB1D1B7819
S11365F0072B03D8BB1D1B78002B01D1992310E076
S1136600BB1D1B78013BDAB2084B1A70FFF7A8FFD9
S1136610FB1D1A787B1D1B78101C191CFEF7ECFA65
S1136620031C181CBD4602B080BDC0460C040020EB
S113663080B500AF044B00221A70FEF789FB031CDF
S1136640181CBD4680BDC0460C04002090B585B022
S113665000AF7860081C111C1A1CFB1C18703B1C32
S11366601980BB1C1A703B1C0F3300221A70284B74
S11366701B78002B05D1FB1C1B78002B01D0952324
S113668041E03B1C0833BA1C12789A703B1C083357
S1136690FA1C12781A703B1C08333A1C1178DC7807
S11366A0002020400143D97052781879002101401C
S11366B00A431A713B1C08333A1C203212785A7070
S11366C07B6819783C1C0F343A1C08323B1C243379
S11366D01B78081C111C1A1CFEF76EFB031C23708C
S11366E03B1C08331B78002B0AD03B1C0F331B7850
S11366F0002B05D1064B1B78013BDAB2044B1A7010
S11367003B1C0F331B78181CBD4605B090BDC0461A
S11367100B04002090B585B000AF7860FB1C1970A5
S1136720BB1C1A703B1C0F3300221A70184B1A78CA
S1136730184B1B789A4205D1FB1C1B78002B01D007
S1136740962320E07B6819783C1C0F34FB1C1A78D4
S1136750BB1C1B78081C111C1A1CFEF743FD031CF0
S11367602370FB1C1B78002B0AD03B1C0F331B78B7
S1136770002B05D1064B1B780133DAB2044B1A7097
S11367803B1C0F331B78181CBD4605B090BDC0469A
S11367900B0400200C04002080B586B000AFF86024
S11367A07A603B1C0B330A1C1A703B1C17333A1CCF
S11367B00B3211780F220A401A703B1C0B331B78E2
S11367C0072B0DD83B1C0B331B78002B08D03B1C2C
S11367D00B331B78013B0F4AD25C7B681A7014E0C0
S11367E03B1C0B331A78102313400CD03B1C17337B
S11367F01B78062B07D83B1C17331B78064AD25C40
S11368007B681A7001E0822300E00023181CBD4657
S113681006B080BDFC0300200404002080B584B0D1
S113682000AF7860FB1C1970BB1C1A703B1C0F3343
S1136830FA1C11780F220A401A70FB1C1B78072BD4
S11368400BD8FB1C1B78002B07D0FB1C1B78013BCF
S1136850334AB91C0978D1545DE0FB1C1A78102323
S1136860134056D03B1C0F331B78062B51D83B1CCE
S11368700E33FA1C1278D2091A70BB1C1B78012B38
S11368800CD179683B1C0F331A783B1C0E331B78F0
S1136890081C111C1A1CFEF713FD32E0BB1C1B78EC
S11368A0002B2ED13B1C0F331B781E4AD35C012BCB
S11368B027D179683B1C0F331A783B1C0E331B78A5
S11368C0081C111C1A1CFEF74BFD3B1C0F331B78D4
S11368D0002B16D13B1C0E331B78013B5A1E9341EF
S11368E0DBB21A1C3B1C0E331A7079683B1C0F3345
S11368F01A783B1C0E331B78081C111C1A1CFEF75B
S11369002FFD3B1C0F331B78064AB91C0978D15460
S113691001E0822300E00023181CBD4604B080BDC2
S1136920FC0300200404002080B582B000AF3A606C
S1136930FB1D021C1A70BB1D0A1C1A700023181CB4
S1136940BD4602B080BDC04680B582B000AF78605D
S11369500A1CFB1C1A70FB1C1B78062B07D9FB1C9A
S11369601B78172B0CD8FB1C1B780F2B08D9FB1C8E
S11369701A78064B9200D358002B01D0002300E074
S1136980C423181CBD4602B080BDC046A4750000D7
S113699080B582B000AF021C3960FB1D1A70FB1D6C
S11369A01B78102B01D1FFF7DBFDFB1D1A78094B77
S11369B09200D358002B07D0FB1D1A78054B920088
S11369C0D3583A68101C98470023181CBD4602B0DF
S11369D080BDC046A475000080B582B000AF786069
S11369E0C046BD4602B080BD002934D00123002238
S11369F010B488422CD301242407A14204D281423A
S1136A0002D209011B01F8E7E400A14204D2814249
S1136A1002D249005B00F8E7884201D3401A1A43C6
S1136A204C08A04202D3001B5C0822438C08A042FD
S1136A3002D3001B9C082243CC08A04202D3001BB3
S1136A40DC082243002803D01B0901D00909E3E72D
S1136A50101C10BC7047002801D00020C04307B4AC
S1136A60024802A14018029003BDC046190000006C
S1136A700029F0D003B5FFF7B9FF0EBC4243891AD1
S1136A801847C0467047C04638B5051C00F0EAFBFD
S1136A9000F090FB084C2368002B02D0984700209C
S1136AA02060064C2168002902D088470022226019
S1136AB0281CF9F7D1FE38BD10040020140400206E
S1136AC010B50023934203D0CC5CC4540133F9E7DE
S1136AD010BD10B5041C00F0EDFA201C10BD00B56B
S1136AE0431E01331A78002AFBD1181A00BD000096
S1136AF0F0B589B001901F1C0EAB03910792029070
S1136B001A78081C01990FAC0138002604922578E4
S1136B100670B14217D1119BB34214D1049B002BD0
S1136B2001D06F2D2FD0642D02D0692D00D0A8E0A4
S1136B30022F02D1039802389FE0012F00D0A0E079
S1136B400398023894E0692D0ED004D8582D16D03D
S1136B50642D1CD108E0752D04D0782D0FD06F2D35
S1136B6015D110E0002712E0019A002A0FDA8024E0
S1136B702606B2420DD051420191029109E000274C
S1136B803E1C102407E000273E1C082403E00026D6
S1136B9000E001260A240090002006900298211C9F
S1136BA0FFF766FF02980591211CFFF71DFF059A68
S1136BB00290092A01D8303205E0059A3732782D3F
S1136BC001D1059A57320098069B02990138D2B236
S1136BD0009002700133002901D00693DEE7011C06
S1136BE0082C0BD10498002808D0302A06D00B1C9E
S1136BF0013B302200931A70069B02330798022847
S1136C000FD1002E01D1002F02D01099013910911B
S1136C10109A1192102C04D10498002801D0023A41
S1136C20119203990098119A091A8918164A9142E7
S1136C3026DC0099CA181199121A8A4203DA01381B
S1136C4030220270F5E7102C0AD1049C002C07D0E6
S1136C50019B002B04D0421E3021023815700170B4
S1136C60002E02D001382D2108E0012F02D1013875
S1136C702B2103E0022F04D101382021017000E010
S1136C80002009B0F0BDC046FD010000F0B5B64CCF
S1136C901E1CA5446B460A900B913E332021002014
S1136CA0197008920590089A1578002D00D1F9E121
S1136CB00898252100F04AFA0C90002811D1089870
S1136CC0FFF70DFF0599021C08180590002A00D152
S1136CD0E8E10B9808990A9EB047002800D0E1E14A
S1136CE0CEE00C9F089C05993A1B8B180593002A4B
S1136CF00CD10C980C9A437801321D1E252D0CD012
S1136D0000270121BC460D97069119E00B980899BC
S1136D100A9DA8470028ECD1B2E00C9A0021023267
S1136D2001240892079106943DE02B2B0BDC202BC9
S1136D3010D0232B00D0BAE001239C4601321378F3
S1136D402B2BF2D1ABE12D2B00D1A5E1302B00D0C0
S1136D50ADE004E00D9D012DF0D00220A0E1069CE1
S1136D60002CEBD002200690E8E737680436FB439A
S1136D70D80F937802321C1C683C0021042C00D8E4
S1136D80C1E0DDB26E2B00D0C7E0013208926E2D57
S1136D9000D149E100D900E1632D00D159E107D8C0
S1136DA0252D00D0F3E010AC25700996012619E0DA
S1136DB0642D00D0EEE0321D09923068032900D022
S1136DC0F6E007996646009601950291039790A90B
S1136DD0069A0D9BFFF78CFE041E00D13FE1634F22
S1136DE06F443E1A069800283CD02023022800D184
S1136DF030236F463E373B7022782B2A04D02D2A4D
S1136E0002D0371C202A0BD1371C302B08D10B9809
S1136E10211C01220A9B9847002831D00134771E97
S1136E20069902290ED1612D01D0412D0AD1012FDD
S1136E3026DD0B98211C02220A9DA84700281FD09A
S1136E40023F0234351C079EB54209DA69460B98A5
S1136E503E3101220A9B9847002811D00135F2E700
S1136E603E1C00E0351C002E03D10698002819D1E1
S1136E7015E0211C0B98321C0A9CA0470028F4D171
S1136E800122554205950DE169463F3120240B98B6
S1136E9001220A9F0C70B8470028F1D00135079FE2
S1136EA0BD42F1DB059A53190593099EFBE6171CB5
S1136EB02A2B00D0E1E0341D36680796002E03DA51
S1136EC073420025079306957B780132261C284FD0
S1136ED00798B84200DDC2E02E2B11D153782A2B3B
S1136EE000D142E7013200271C1C303C092C05D894
S1136EF00A214F4301323F191378F5E701203AE79D
S1136F000027381C37E71B4D295D1B4D2C57002CDF
S1136F1000D136E75378013233E76E2B0ADC632B5A
S1136F202CD002DC582B30D115E0642B13D0692B04
S1136F302BD110E0732B23D009DC6F2B0BD0702BDB
S1136F4023D101237825082703219C461DE7752BAF
S1136F5001D0782B19D1002815D0069C022C00D022
S1136F6013E70123069310E7BCFDFFFF3F02000077
S1136F70FD0100000A76000005760000002804D117
S1136F80002902D101E70127FFE6FF25FDE6582D80
S1136F9065D116E0692D62D10DE7732D23D002D897
S1136FA06F2D5CD10DE0752D0BD0782D57D108E0F5
S1136FB0022901D100B204E7012900D001E740B25F
S1136FC0FFE6341D09943068032906D0022901D153
S1136FD080B202E0012900D1C0B2079E624600924D
S1136FE001950296F2E63468311D0991002C00D116
S1136FF02F4C6346002B07D026780134002800D19B
S1137000F0E6BE4237DCEDE6002808D0201C6146DD
S11370103A1C00F08EF800282DD0061BE2E6201C56
S1137020FFF75DFD061CDDE6351D09953468022970
S113703007D003290AD0002900D036E7059820603C
S113704033E76F461421CB5B23802EE7059A226039
S11370502BE73368301D10AC09902370A6E60C981A
S1137060FFF73DFD059E021C35180595002819D033
S11370700B980C992FE63E1CB4E600240794191CC7
S11370803039092900D922E7079D0A236B430132CD
S1137090581807901378F2E7002706974EE6012068
S11370A00D904BE605989124A400A544F0BDC0467C
S11370B00476000030B5C9B2031C1F2A31D94442FA
S11370C00323234005D0D21AC51801700130A84209
S11370D0FBD1002905D00D060C042C430B022143DF
S11370E019435409031C002C0ED0251C013D1960C2
S11370F059609960D960196159619961D9612033E6
S1137100002DF3D16301C318D006400F07D0041C2F
S11371101D1C013C02C5002CFBD180001B1803245C
S113712022409D18002A03D019700133AB42FBD1D1
S113713030BD00B5C9B28218904205D00378013041
S11371408B42F9D1013800E0002000BD00B5C9B27E
S11371500378421C002B03D08B4205D0101CF7E7A8
S11371604B4259414942084000BD000010B50B4C48
S11371700B4B9C4202D001CC8047F9E7094C0A48EA
S1137180844202D008CC9847F9E7084C08498C425D
S113719002D004CC9047F9E710BDC0461076000039
S11371A010760000107600001076000010760000C3
S11371B01076000010B5084C084B9C4202D004CC59
S11371C09047F9E7064C0748844203D0043C216801
S11371D08847F8E710BDC04610760000107600001E
S11371E0107600001076000000B588421FD0002AF7
S11371F01DD00323194207D1184205D19A4203D95D
S113720008C9043A08C0F2E70123194209D1184217
S113721007D19A4205D90B88023A03800231023021
S1137220E5E70B78013A037001310130DFE700BD77
S113723038B50B4D002D11D000242B1919680029E5
S113724006D02B1958689A68FFF7CEFF0C34F4E780
S11372505A68002AF5D198680028F2D138BDC04692
S1137260F8760000054B10B51C68002C04D0A0680B
S1137270616888472468F8E710BDC04624040020EC
S1137280054B181C002805D0854681B00020C0435A
S1137290009001B0F746704700000020F7467047A1
S11372A08001020303010201100002020010000326
S11372B00301100000001200200000000000000084
S11372C0000000000000000004F0FF1F18F0FF1F82
S11372D000000000000000000000000000000000AA
S11372E000000000043A242238F0FF1F3CF0FF1F86
S11372F078F0FF1F9CF0FF1F38F0FF1F0400000010
S113730009040000E8720000E472000000000000BC
S1137310000000000000000000010000BE22000088
S1137320C6220000CE220000D6220000DE22000089
S1137330E6220000EE220000DA250000E22500002B
S1137340EA250000F2250000FA25000002260000CC
S11373500A260000562900009E2900009E290000EC
S11373609E2900009E2900009E2900009E290000FD
S11373709E2900009E2900009E2900005E2900002D
S11373809E2900009E2900009E2900009E290000DD
S11373909E2900009E2900009E2900009E290000CD
S11373A09E290000662900009E2900009E290000F5
S11373B09E2900009E2900009E2900009E290000AD
S11373C09E2900009E2900009E2900006E290000CD
S11373D09E2900009E2900009E2900009E2900008D
S11373E09E2900009E2900009E2900009E2900007D
S11373F09E290000762900009E2900009E29000095
S11374009E2900009E2900009E2900009E2900005C
S11374109E2900009E2900009E2900007E2900006C
S11374209E2900009E2900009E2900009E2900003C
S11374309E2900009E2900009E2900009E2900002C
S11374409E290000862900009E2900009E29000034
S11374509E2900009E2900009E2900009E2900000C
S11374609E2900009E2900009E2900008E2900000C
S11374709E2900009E2900009E2900009E290000EC
S11374809E2900009E2900009E2900009E290000DC
S11374909E29000096290000FA2A0000122B000001
S11374A02A2B0000422B00005A2B0000722B0000F4
S11374B0843400008C34000094340000AE340000A6
S11374C0C83400006C3500006C3500006C350000D9
S11374D06C3500006C3500006C3500006C35000024
S11374E06C3500006C3500006C3500006C35000014
S11374F06C3500006C3500006C3500006C35000004
S11375006C3500006C3500006C3500006C350000F3
S11375106C3500006C3500006C3500006C350000E3
S11375206C3500006C3500006C3500006C350000D3
S11375301C350000023500003635000050350000CF
S11375400101000101000000000101000000000031
S1137550010101010100000001010001010001001D
S11375600001000001000000853C0000493E0000CD
S113757000000000493E00000000000051400000EF
S11375801D43000000000000D54000002941000018
S11375900542000069420000C542000008000000E6
S11375A004000000E939000065300000E531000006
S11375B0192F0000D9690000D9690000D9690000B9
S11375C0D9690000D9690000D9690000D9690000AF
S11375D0D9690000D9690000D9690000D96900009F
S11375E0D9690000E5440000A1430000694400009B
S11375F0E5430000A1430000D9690000FD450000F7
S113760035440000000100000001020000000300F6
S1137610010000001201000200000010A215170072
S1137620000201020001000009022000010100C063
S1137630320904000002FF00FF0007058102100068
S11376400007050202100000040309043A0346007F
S11376507200650065007300630061006C006500E2
S11376602000530065006D00690063006F006E0028
S113767064007500630074006F007200200049000C
S11376806E0063002E0000002403550053004200E6
S1137690200074006F0020005300500049002000B7
S11376A0440065007600690063006500220342001F
S11376B041004400200053005400520049004E0091
S11376C04700200049004E004400450058000000D7
S11376D000C20100000008000000000000000000DB
S11376E004000000C0D40100A1200000000002003A
S10B76F000000000FF0000008F
S11376F81076000000F0FF1FE8000000F876000094
S1137708000000200000000000000000000000004D
S10777180000000069
S9030829CB
